:02000004000FEB
:1010000020C90020DD130F00E5130F00E7130F00C8
:10101000E9130F00EB130F00ED130F0000000000A9
:10102000000000000000000000000000C9130F00D5
:10103000F1130F0000000000F3130F00F5130F0071
:10104000F7130F00F7130F00F7130F00F7130F003C
:10105000F7130F00F7130F00F7130F00F7130F002C
:10106000F7130F00F7130F00F7130F00F7130F001C
:10107000F7130F00F7130F00F7130F00F7130F000C
:10108000C12C0F00712A0F00F7130F00F7130F0088
:10109000F7130F00F7130F00E12A0F00F7130F00EB
:1010A000F7130F00F7130F00F7130F00F7130F00DC
:1010B000F7130F00F7130F000000000000000000FE
:1010C000F7130F00F7130F00F7130F00F7130F00BC
:1010D000F7130F00F7130F00F7130F00F7130F00AC
:1010E000F7130F00F7130F00C5150F0000000000E5
:1010F00000000000F7130F0000000000F7130F00BE
:1011000000000000000000000000000000000000DF
:1011100000000000000000000000000000000000CF
:1011200000000000000000000000000000000000BF
:1011300000000000000000000000000000000000AF
:10114000000000000000000000000000000000009F
:10115000000000000000000000000000000000008F
:10116000000000000000000000000000000000007F
:10117000000000000000000000000000000000006F
:10118000000000000000000000000000000000005F
:10119000000000000000000000000000000000004F
:1011A000000000000000000000000000000000003F
:1011B000000000000000000000000000000000002F
:1011C000000000000000000000000000000000001F
:1011D000000000000000000000000000000000000F
:1011E00000000000000000000000000000000000FF
:1011F00000000000000000000000000000000000EF
:10120000DFF80CD000F0A0F90048004755540F005B
:1012100020C9002080F308888E46104730B450E87B
:10122000012F93B2C48923448489A34228BF1B1B86
:101230000489A34202BFBFF32F8F002007E0C3EA57
:10124000020340E80134002CE9D14FF001000A60AC
:1012500030BC704750E8012FC2EA024240E8012149
:101260000029F7D1704730B450E8022F1FFAA2F3DB
:10127000C488A34202BFBFF32F8F00200DE0C489B2
:1012800023448489A34228BF1B1BC2EA034340E8CE
:101290000234002CE8D14FF001000A6030BC7047E6
:1012A00050E8022FC2EA224240E802210029F7D189
:1012B0007047034653E8022FD988B2EB324F4FF004
:1012C000000017BF92B241EA014142EA014104E045
:1012D0005A68B2EB324F08BF012043E80212002ADD
:1012E000E8D1704730B4044654E8000F0D4644E896
:1012F0000053002BF8D1156030BC704730B4044661
:1013000054E8000F40EA010544E80053002BF7D1F0
:10131000156030BC704730B4044654E8000F00EA52
:10132000010544E80053002BF7D1156030BC70472D
:1013300030B4044654E8000F80EA010544E8005345
:10134000002BF7D1156030BC704730B4044654E828
:10135000000F00EB010544E80053002BF7D11560A6
:1013600030BC704730B4044654E8000FA0EB0105D0
:1013700044E80053002BF7D1156030BC704770B4BF
:1013800004464FF0000054E8006F0D68AE4207BFFE
:1013900044E80023012044E800630E60002B1CBFDA
:1013A0000020F0E770BC704730B4044654E8000FEA
:1013B00088422CBF451A054644E80053002BF5D15E
:1013C000156030BC704700001EF0040F0CBFEFF337
:1013D0000880EFF3098007F0B7BE00000648804799
:1013E00006480047FEE7FEE7FEE7FEE7FEE7FEE70A
:1013F000FEE7FEE7FEE7FEE7E52A0F0001120F0019
:101400002DE9F05F0546002092469B468846064639
:10141000814640241BE0284641464746224600F0CC
:1014200083F853465A46C01A914110D311461846C4
:10143000224600F016F82D1A67EB01084F462246A7
:101440000120002100F00DF817EB00094E41201E8D
:10145000A4F10104DFDC484631462A464346BDE894
:10146000F09F202A04DB203A00FA02F100207047A6
:101470009140C2F1200320FA03F3194390407047D2
:101480000048704754BD0F0010B5441A03469442FB
:1014900009D28418114403E011F8013D04F8013D1C
:1014A000521EF9D210BD40EA0104A40703D009E09E
:1014B00010C9121F10C3042AFAD203E011F8014B1D
:1014C00003F8014B521EF9D210BDD2B201E000F870
:1014D000012B491EFBD270470022F6E710B51346D8
:1014E0000A4604461946FFF7F0FF204610BD421C8D
:1014F00010F8011B0029FBD1801A704730B5044653
:101500000020034600E05B1C934203D2E05CCD5C0C
:10151000401BF8D030BD034611F8012B00F8012B19
:10152000002AF9D118467047202A04DB203A21FA14
:1015300002F00021704721FA02F3D040C2F12002EC
:101540009140084319467047064C074D06E0E06895
:1015500040F0010394E8070098471034AC42F6D3FA
:10156000FFF752FE08CD0F0028CD0F0070B58C1884
:1015700010F8015B15F0070301D110F8013B2A11A7
:1015800006D110F8012B03E010F8016B01F8016B94
:101590005B1EF9D12B0705D40023521E0DD401F890
:1015A000013BFAE710F8013BCB1A921C03E013F859
:1015B000015B01F8015B521EF9D5A142D8D300208E
:1015C00070BD0000054B4FF0FF321A6053F8042C39
:1015D000034B1A601A68034B1A60704704BA025032
:1015E00018A9002008BA025001EB820204388A428E
:1015F00001D10020704752F8043D1BBA40F8043F67
:10160000F5E7000000B5374B8FB019461A68009215
:10161000009AD207FAD5344B344A1A600A6801920C
:10162000019AD007FAD5324A1A600A680292029AE1
:10163000D207FAD52F4A1A600A680392039AD00794
:10164000FAD52D4A1A600A680492049AD207FAD58C
:101650002A4A1A600A680592059AD007FAD5284ADC
:101660001A600A680692069AD207FAD5254A1A60C5
:101670000A680792079AD007FAD5234A1A600A68BF
:101680000892089AD207FAD5204A1A600A68099285
:10169000099AD007FAD51E4A1A600A680A920A9A6D
:1016A000D207FAD51B4A1A6008680B900B98C0073E
:1016B000FAD51A600A680C920C9AD007FAD5164A25
:1016C0001A600A680D920D9AD207FAD5134A1A6069
:1016D0000E210D230F22002000F088FD0FB05DF8D1
:1016E00004FB00BFB0B0025080B00250804301291B
:1016F00040633921807001298020542100D1349029
:10170000C0403490C0302029C0530D900041389023
:10171000832308C880E3102100413821CF4308C843
:1017200010B5504B96B01C461A680192019AD20728
:10173000FAD54D4B4D4A1A6022680292029AD2079E
:10174000FAD54B4A1A604B4A42EA8040226803921B
:10175000039AD207FAD5186022680492049AD00737
:10176000FAD5454A1A60A2F5800242EA8141226810
:101770000592059AD207FAD5196022680692069A50
:10178000D007FAD53D4A1A6022680792079AD10716
:10179000FAD53B4A1A6022680892089AD207FAD50D
:1017A000384A1A6022680992099AD007FAD5364A4F
:1017B0001A6022680A920A9AD107FAD5334A1A6047
:1017C00022680B920B9AD207FAD5314A1A60226826
:1017D0000C920C9AD007FAD52E4A1A6022680D9204
:1017E0000D9AD107FAD52C4A1A6022680E920E9AE9
:1017F000D207FAD5294A1A6022680F920F9AD007A9
:10180000FAD5274A1A60216810911099C907FAD5AC
:101810001A60144B1A46196811911199C807FAD524
:10182000114B20491960116812911299C907FAD514
:101830001D491960116813911399CC07FAD50B490A
:101840001960116814911499C807FAD517491960DD
:10185000116815911599C907FAD5154A1A6016B07D
:1018600010BD00BFB0B0025080B0025040044190A3
:1018700000862929D81001C840144190401421291C
:10188000401465210034409000310C90C0400C9011
:10189000C030202940960D9000416090031645C845
:1018A0000086112100416021594644C840144590EA
:1018B00040142D90F0B5464B89B01D461C6801942C
:1018C000019CE407FAD5434BDFF810C1DFF810E1C3
:1018D00013449B000A181B681E2A88BFC0F11E0112
:1018E0001F330A185B095A43B2F5806F88BF4FF463
:1018F00080614FF0000484BFB1FBF3F1091A00F1DD
:10190000A05000F52C402746A14233DC2A680492FF
:10191000049AD207FAD5304A1268296805910599C8
:10192000CF07FAD52D482E4C0260002216469A4267
:1019300002F1010140D12A4C134621F00101002699
:101940008B423CD32B680693069BDE07FAD5254BCA
:101950001B682C680794079CE407FAD503600023F2
:101960001F481C469A422DD11D4A00208B422CD381
:1019700009B0F0BD2A680292029AD207FAD502197C
:10198000920012682E680396039EF607FAD5CCF8EB
:10199000002000229A4202F1010206D11E4622F0E6
:1019A0000102964204D30134AEE7CEF80070F1E7AD
:1019B000CEF800700136F4E726600A46B7E72660E5
:1019C0000133BDE704600133CCE710600133CDE79C
:1019D000B4B0025024AC00147CB00250D4B0025019
:1019E000D8B0025078B00250F0B5294D85B02C46E1
:1019F0002E680096009EF607FAD500F1A05000F57B
:101A00002C4080000568206801900198C707FAD52E
:101A10002048214F056002EB8306B24229D15A1CAF
:101A20001D4E22F001020027934227D32368029320
:101A3000029BDE07FAD5194B0B449B001B681F3332
:101A40005B099A4213D2216803910399C907FAD519
:101A5000154400219B1A104A05600846994210D38C
:101A60005A1C0D4922F00102002093420CD305B00C
:101A7000F0BD52F804EBC7F800E0CEE73760013361
:101A8000D2E710600131E9E708600133EDE700BFFC
:101A9000B4B00250D4B00250D8B0025024AC0014FC
:101AA00010B5494B94B019461A680092009AD207B3
:101AB000FAD5464B464A1A600A680192019AD40741
:101AC000FAD5444A1A600A680292029AD007FAD5F7
:101AD000414818600A680392039AD207FAD53F4A30
:101AE0001A600A680492049AD407FAD53C4A1A602C
:101AF0000A680592059AD207FAD53A4A1A600A6826
:101B00000692069AD407FAD5374A1A600A680792ED
:101B1000079AD207FAD5354A1A600A680892089AD5
:101B2000D407FAD5324A1A600A680992099AD2078C
:101B3000FAD5304A1A600A680A920A9AD407FAD586
:101B40002D4A1A600A680B920B9AD207FAD52B4AD3
:101B50001A600A680C920C9AD407FAD5284A1A60BF
:101B60000A680D920D9AD207FAD5264A1A600A68B9
:101B70000E920E9AD407FAD5234A1A600A680F9279
:101B80000F9AD207FAD5214A1A600F4B19461C68E2
:101B90001094109CE407FAD50C4B1860086811905B
:101BA0001198C407FAD51A600A681292129AD007DF
:101BB000FAD5174A1A600A681392139AD207FAD50F
:101BC000144A1A6014B010BDB0B0025080B0025078
:101BD0008090652100040990409665908080612185
:101BE00080200821802064900081619000461021AF
:101BF000008111210041442180202029024610C883
:101C000000860921802060214021282940966521F5
:101C100040962529594614C810B5544B98B019461A
:101C20001A680192019AD207FAD5514B514A1A60AB
:101C30000A680292029AD407FAD54F4A1A600A68D3
:101C40000392039AD007FAD54C4818600A680492A8
:101C5000049AD207FAD54A4A1A600A680592059A88
:101C6000D407FAD5474A1A600A680692069AD2073C
:101C7000FAD5454A1A600A680792079AD407FAD536
:101C8000424A1A600A680892089AD207FAD5404A6E
:101C90001A600A680992099AD407FAD53D4A1A606F
:101CA0000A680A920A9AD207FAD53B4A1A600A6869
:101CB0000B920B9AD407FAD5384A1A600A680C922C
:101CC0000C9AD207FAD5364A1A600A680D920D9A14
:101CD000D407FAD5334A1A600A680E920E9AD207D0
:101CE000FAD5314A1A600A680F920F9AD407FAD5CA
:101CF0002E4A1A600A681092109AD207FAD52C4A16
:101D00001A601A4B19461C681194119CE407FAD505
:101D1000174B1860086812901298C407FAD51A6019
:101D20000A681392139AD007FAD5124A1A600A6801
:101D30001492149AD207FAD51E4A1A600A681592AC
:101D4000159AD407FAD51C4A1A600A681692169A90
:101D5000D007FAD5194A1A600A681792179AD2075B
:101D6000FAD5174A1A6018B010BD00BFB0B00250C3
:101D700080B0025000936521000431904096659038
:101D80000083612100C3302100C364900081619011
:101D900000461021008111210041442100C3202967
:101DA0000C4610C80086312100C3602140C128299B
:101DB000409665210013319040962529594614C854
:101DC000400432492DE9F041814B1D689868203369
:101DD000A0B01E461A680192019AD707FAD57D4B2A
:101DE0007D4A1A6032680292029AD407FAD57B4A79
:101DF0001A607B4A1446116803910399C907FAD502
:101E0000784A1168C1F3402137680497049FFF079F
:101E1000FAD5754F1F6027680597059FFF07FAD50C
:101E20001768002900F0CF80B90540F1CC803168F7
:101E300006910699CF07FAD56C4919602168079178
:101E40000799C907FAD51168C1F340213768089787
:101E5000089FFF07FAD5664F1F6027680997099FFB
:101E6000FF07FAD51268002900F0AF80910540F114
:101E7000AC8032680A920A9AD207FAD5564A1A609A
:101E800032680B920B9AD707FAD55A4A1A60316812
:101E90000C910C99CC07FAD55749196031680D910E
:101EA0000D99C907FAD55549196031680E910E99F7
:101EB000CF07FAD55249196031680F910F99CC07B5
:101EC000FAD550491960504B1E4619681091109967
:101ED000C907FAD53F4C4D4B236033681193119BD2
:101EE000DB07FAD54A4B236033681293129BDF0756
:101EF000FAD5484B23603A4B9846196813911399C9
:101F0000C907FAD5324F386033681493149BDB0746
:101F1000FAD5226033681593159BD807FAD53E4B46
:101F2000236033681693169BD907FAD53B4B236081
:101F300033681793179BDA07FAD5394B2360336858
:101F40001893189BDB07FAD5364B23603368199337
:101F5000199BD807FAD5344B236033681A931A9B20
:101F6000D907FAD5314B236033681B931B9BDA07E3
:101F7000FAD52F4B236000F0D3F908BBD8F8003016
:101F80001C931C9BDB07F9D53D6033681D931D9B9B
:101F9000D907FAD5274B236033681E931E9BDA07B7
:101FA000FAD5254B2360D8F800301F931F9BDB0721
:101FB000F9D50C4B1B6813F4805F204B08BF184603
:101FC00020B0BDE8F0811E48FAE71E48F8E700BFE0
:101FD00090B0025080B0025000100251C01F722910
:101FE000B4B0025088B00250C0CF0129C01F0E29E2
:101FF000C03F002940010249003184A80000164971
:10200000400108A180440888B0B00250C0447088E4
:1020100080077A41C0077E4100006A498006164960
:1020200040006E49000200210082202140822021D0
:102030008082242140A161A100C861510308F10000
:102040000108F1000208F10008B540B1202801465E
:102050004FF0070228BF20210020FFF72BFC024B86
:1020600000221A6008BD00BF1CB802507FB51C6872
:102070001CB901F01F041F2C27D1174C25462668D8
:102080000196019EF607FAD500F1A05000F52C400C
:10209000800000682C680394039CE407FAD50F4C79
:1020A00000EB611020600E4801F01F0400680290F0
:1020B0001F2C18BFC94302980FBF106001F01F0109
:1020C00000FA01F111600021196010684300C00F8F
:1020D000136004B070BD00BFB4B00250E4B0025051
:1020E000DCB0025030B51E4B85B01A46196800911D
:1020F0000099CC07FAD500F1A05000F52C408000E3
:10210000016813680193019BD807FAD5154B164C4B
:102110001868164D1F30202390FBF3F0013800287B
:1021200010DA00230130400153B1A0F120014FF03B
:102130000042134204D1013881424FEA5202F8D1E1
:1021400005B030BD13680393039BDB07FAD5431832
:1021500023602B680293029B002BE3D10138DEE75A
:10216000B4B00250ACB00250E4B00250DCB0025047
:102170000A460021AFF3008038B5A0F12003B3F583
:10218000426F05462CD88F2826D800F1470300F16E
:102190006604DB064FEA541400D0013464013F3476
:1021A000A409013411B1A1421AD30C46E3004FF443
:1021B0008050B0FBF3F0202828BF202002B110602F
:1021C000084B01221A60214600F068F82846214693
:1021D00000F088F8002038BD00F11F046409DDE735
:1021E000014838BD1CB802502221F00070B52648C5
:1021F00088B0054604680094009CE607FAD5234899
:10220000234C0460234C44EA83432C680194019CD2
:10221000E407FAD50360930143EA824242F0104496
:1022200044F4C0442B680293029BDE07FAD5046095
:102230002B680393039BDB07FAD5174B03608B01D5
:1022400043EA814141F0104343F4C0432E680496B1
:10225000049EF607FAD503602B680593059BDE07FD
:10226000FAD5046041F058412B680693069BDC07C1
:10227000FAD5016042F058422B680793079BDB07B1
:10228000FAD5026008B070BDB0B0025080B0025004
:10229000C0210229807100988061189030B5002219
:1022A0000C4C49001346023840F6FC75904202F18E
:1022B0000102CABF236025605B181E2A04F10404D2
:1022C000F4D1054A19441360044B054A19609A6019
:1022D00030BD00BF00B0025078B002507CB0025058
:1022E00020F80F000C4B18603F3020F03F008901B0
:1022F000403058609960D9601961596199611C3307
:102300000648196082B002680192019AD207FAD594
:10231000196002B0704700BF90B00250B4B00250D4
:102320002DE9F04192B0012303930493624B1D46C3
:102330001A680592059AD207FAD5604C604B236063
:10234000604B19461A680692069AD707FAD55E4B73
:102350001A68D60400F1A8802A680792079AD00765
:10236000FAD55A4A22600A680892089AD207FAD522
:102370001E68C6F30036002E40F098801220FFF74A
:10238000B1FE07461320FFF7ADFE87428CBF122037
:102390001320FFF7A7FE471EFFF734F903AB01AA8E
:1023A00039461220FFF762FE04AB804602AA394686
:1023B0001320FFF75BFE00EB4800022832D0032811
:1023C0003ED0012874D12B680993099BDB07FAD50D
:1023D0003F4B23602B680A930A9BD807FAD53D4BE5
:1023E00023602B680F930F9BD907FAD53A4B2360D4
:1023F0002B681093109BDA07FAD5384B23602B68B3
:102400001193119BDB07FAD5354B2360013F25D58E
:102410001023192218210020FFF7E8FE304612B0E1
:10242000BDE8F0812B680B930B9BD907FAD52D4B98
:1024300023602B680C930C9BDA07FAD52A4BCFE765
:102440002B680D930D9BDB07FAD5284B23602B6877
:102450000E930E9BD807FAD5254BC1E703AB01AA13
:1024600039461220FFF702FE04AB044602AA3946A1
:102470001320FFF7FBFD10EB440402D1FFF7CCFB68
:10248000C4E7FFF70DFB022C08D0032C09D0012C68
:1024900010D117211620FFF743F9B7E715211420B3
:1024A000F9E70F210E20F6E7124EB7E7124EB5E717
:1024B000124EB3E7124EB1E7B0B0025080B00250F6
:1024C00000084A51B4B0025088B0025000084E5182
:1024D00000065A4940065E49000442410014424940
:1024E00040042E49000652494006564900063A4922
:1024F00040063E490608F1000708F1000408F10013
:102500000508F100014B1860704700BF08BA02507F
:10251000014B1860704700BF04BA0250094BC24318
:102520001A60043B82B01B680193074B019A10426A
:1025300004D0064A1060186802B0704720BF1A68BD
:102540000192F3E704BA025018A9002008BA025019
:10255000FEF79ABFFEF7C2BF0A460021FEF7BEBFD4
:102560002DE9F74305460E469946114600F060FAFC
:102570000446002840F08480002E00F08580002969
:1025800000F08480B9F1200F40F0828005F144040E
:10259000082205F104082046FFF726F805F1240774
:1025A000082231464046FFF71FF806F120010822B5
:1025B0003846FFF719F802A94FF4807041F8049DDE
:1025C000FFF7D6FD002865D1334A4FF480731360BE
:1025D000012193600823314AFFF706FA01210846DA
:1025E00005232F4AFFF700FA0823424601211C2049
:1025F000FFF7FAF908233A4601210320FFF7F4F91F
:102600002246082301210220FFF7EEF90823254A7C
:1026100001211A20FFF7E8F90523234A01211B2095
:10262000FFF7E2F90823214A01211420FFF7DCF922
:1026300008231F4A01211520FFF7D6F9082305F1C9
:10264000640201211620FFF7CFF9082305F1840267
:1026500001211720FFF7C8F90823164A01210B2092
:10266000FFF7C2F9FFF7AEFB04460198FFF7ECFC59
:10267000114B002C18BF1C46A4212846FFF76CFF05
:10268000204603B0BDE8F0830C4CF9E70C4CF7E7AB
:102690000C4CF5E7084CEFE790B002507CCC0F00F3
:1026A000F4CC0F003CCC0F00E0CC0F00A0CC0F000E
:1026B000C0CC0F005CCC0F008408F0007608F0005E
:1026C0008008F0008108F00038B50D460446B0B12E
:1026D000A02200210430FFF73DFF95B129460822D2
:1026E00004F16400FEF780FF082205F1200104F1E7
:1026F0008400FEF779FF044B2360002038BD0348B7
:1027000038BD034838BD00BFDD55AABB7108F000D5
:102710008308F0002DE9F041069F044615461E4649
:10272000FFF7D2FF38B93B46324629462046BDE87E
:10273000F041FFF715BFBDE8F08100002DE9FF4132
:10274000144B04460E460FCB8DE80F00204600F0D8
:102750007FF98046B0B9CEB1636A251D01953BB9BA
:1027600001236362226F04F13001684600F088F8AB
:102770002B46043E243453F8042B12BAA34246F8E5
:10278000042FF8D1404604B0BDE8F081DFF808809E
:10279000F8E700BF0CCC0F000502F00038B5044686
:1027A00068B1051D28467021FFF7D6FE2846202275
:1027B0000449FFF7CDFE044B2360002038BD0348D9
:1027C00038BD00BF1CCC0F00DD55AABB0002F000D5
:1027D000294B2DE9F04304460E4615460FCB85B034
:1027E0006F468DE80F002DB94FF00009484605B03F
:1027F000BDE8F083204600F02BF981460028F5D192
:10280000231D0193636AA3BB236F8BB1C3F14008FF
:10281000A84528BFA84604F1300031461844424676
:10282000FFF796FE236F434446442367A5EB080554
:10283000226F402A06D104F13001384600F020F81A
:102840000023236705F03F0835F03F0505D03146EA
:102850002A46384600F014F82E44B8F1000FC3D0D1
:102860004246314604F13000FFF772FEC4F8708032
:10287000BCE7DFF80890B9E70CCC0F000C02F000C1
:102880002DE9F74F314B44688046924699461A68C5
:10289000002AFCD12E4B9B461A68002AFCD14FF02F
:1028A000FF300191FFF72EFE8020FFF731FE294D0A
:1028B000294A2A4F2A4E012307202B60A2F59E7237
:1028C000C2F83C011360636A3B60A36A3360D8F8C6
:1028D000003042F8043CD8F8083020469847019967
:1028E000D9F80030002BFBD1BAF1000F20D11D4BDD
:1028F00004221A60D9F80030002BFBD1DBF800A0CD
:10290000BAF1000FFAD1D8F80C30204698473B684E
:1029100063623368A362144BC3F800A0C3F844A1F8
:10292000D9F80030002BFBD12B6003B0BDE8F08F4D
:10293000236A012B04BF0C4A13600C4B4020196022
:10294000C3F804A0FFF7EAFDD4E700BF10B90250B6
:1029500020BC025018B8025000B90250CCB7025047
:10296000D0B70250C8B7025084B6025028BC0250FB
:10297000084B1B681B0EF02B08D1074B1A68074B3E
:102980009A4205D1064B0020186070470520704719
:102990000620704728B9025024BA02500000E020F7
:1029A0000CBA02500C4B1B68C3610C4B1B68836153
:1029B0000B4B1B6843610B4B1B6803610A4B1B6885
:1029C000C3600A4B1B688360094B1B684360094B5B
:1029D0001B680360704700BF5CB6025058B60250D7
:1029E00054B6025050B602504CB6025048B602508F
:1029F00044B6025040B602500C4BC2691A6082695C
:102A000043F8042C426943F8082C026943F80C2C63
:102A1000C26843F8102C826843F8142C426843F8CB
:102A2000182C026843F81C2C704700BF5CB602509B
:102A300030B10268034B04489A4208BF0020704737
:102A400002487047DD55AABB8208F0007108F0000B
:102A500030B10268034B04489A4208BF0020704717
:102A600002487047DD55AABB0202F0000002F000E8
:102A700002490248091F0968006808478058002079
:102A800000F02EB970B50E46144900EB400001EB82
:102A9000C0051446E86A183520B101280FD0022875
:102AA00005D113E0284600F051F9A04201D20024DC
:102AB00011E022463146284600F080F90BE0284616
:102AC00000F044F9A042F4D20446F2E73146284629
:102AD00000F047F90446204670BD000090980020A1
:102AE00006F040B930B54FF0805000228300D0F896
:102AF0003011C3F80C21C3F81021624B1A60624BED
:102B00001B68624C2360604B1B1D1B68241D2360E7
:102B10005D4B08331B68241D23605B4B0C331B6823
:102B2000241D2360584B10331B68241D2360564B13
:102B300014331B68241D2360534B18331B68534CFC
:102B400020342360504B1C331B68241D23604E4BE4
:102B500020331B68241D23604B4B24331B68241D2A
:102B60002360494B28331B68241D2360464B2C33BC
:102B70001B68241D2360444B30331B68434C403496
:102B80002360414B34331B68241D23603E4B383394
:102B90001B68241D23603C4B3C331B68241D2360B1
:102BA000394B40331B68241D23600124082902D1BE
:102BB000D0F8343113B1082904D006E0354B34493C
:102BC000196005E0D0F8343113B1082904D006E0CB
:102BD000314BFB21196005E0D0F8343113B10829DD
:102BE00008D00EE090F858322C48016863F30301D6
:102BF000016002E0D0F834311BB929494FF400706C
:102C0000086028480168C90702D06FF0010101601F
:102C10002548016841F470010160BFF34F8FBFF395
:102C20006F8F4FF01021D1F80002002803DBD1F89C
:102C30000402002822DA1D4B1C601D480468002C89
:102C4000FCD01224C1F800420568002DFCD0C1F868
:102C5000044201680029FCD01A6001680029FCD0F8
:102C6000BFF34F8F10487C380168124A01F4E061CD
:102C700011430160BFF34F8F00BFFDE70F490E48BE
:102C8000086030BD380500400404001020C5004035
:102C9000488103008C56004018F50040E40E0040C7
:102CA000409602400004004088ED00E004E5014049
:102CB00000E401400400FA050090D0030C59002004
:102CC000064808B5002101600068009005F054FD39
:102CD00005F020FB0028FBD108BD000000010140E9
:102CE00010B5124C02202061606111A0A06104F1B6
:102CF0007800E0614FF4805020620020A0626062A2
:102D00000BA1A164E0620D49E1641021A065C4E952
:102D10001410E0650AA1E01DFEF7FDFB09A12046A5
:102D2000FEF7F9FB2020A07110BD00009098002054
:102D30005465726D696E616C0000000008A9002086
:102D40005254540053454747455200000269C16838
:102D50008A4203D88068401A104400E0501A401E8E
:102D600070472DE9F047C4681746894606464FF07C
:102D700000083069A04201D9051B02E0B168201AA1
:102D80000D1AB0686D1E001BA84200D80546BD4252
:102D900000D33D4670682A4620444946FEF774FB3E
:102DA000B0687F1B2C44A844A944A04200D1002451
:102DB000F460002FDDD14046BDE8F0872DE9F041F9
:102DC00004468846D4E90207C51BE16860681646D8
:102DD0000844B54206D94146FEF756FBB819E060F3
:102DE000BDE8F0812A464146FEF74EFB761B08EB14
:102DF000050132466068FEF747FBE660F0E702E057
:102E000008C8121F08C1002AFAD170477047002075
:102E100001E001C1121F002AFBD1704701212028C7
:102E200003DA81400548014003E0402802DA2038F7
:102E3000814009B10120704700207047FC06FFBDAA
:102E4000800701D00020704701207047406800686B
:102E5000401E084201D10120704700207047C3681E
:102E60008B4206D811440069491E814201D80120D5
:102E7000704700207047000030B585B00D46164CF5
:102E80001621ADF800101ECC0DF1040C8CE81E00CC
:102E9000124C0221012221706270A0700320E070A8
:102EA000217159206071FE20A071694604F109006A
:102EB0007DDF00280ED1BDF800002A46411CE171DB
:102EC00009212172BDF808100844ADF8080001A9D5
:102ED000034872DF05B030BD00B90F009C6D0020C3
:102EE0000858002010B586B0062418220C49684600
:102EF000FEF7CAFA0B480421008801EB00400AA142
:102F000005F06CFB69462046FFF7B6FF002805D1A7
:102F1000094C207874DF0121207873DF06B010BDE2
:102F200010B90F00305900204164766572746973DE
:102F3000696E672E2E2E0000085800202DE9F05FE4
:102F4000DFF894B05C46DBF84890DBF8245003F0DF
:102F500045FA216B214E00EB01086F1A31884FF0C2
:102F6000040A0AEB01401EA105F038FB216B404624
:102F70004944414500D1002708233A4601F0F8FFB3
:102F800007004FF0010806D0318808EB01401BA173
:102F900005F024FB1CE003F021FA0022294601F091
:102FA00009FADBF8282004463188D946A24209D123
:102FB0000AEB014018A105F011FBC9E90748C9F85F
:102FC000185005E008EB01402346194905F011FBB4
:102FD0003846BDE8F09F0000EC7F00206C590020CF
:102FE000456E746572206E72665F6466755F6170AF
:102FF000705F636F6E74696E756500004661696C21
:10300000656420746F20636F7079206669726D77D4
:103010006172652E0000000053657474696E67204C
:103020006170702061732076616C6964000000003B
:10303000F4BD0F0008B5134602460648009301236D
:10304000008803EB00400B4603A105F0DAFA06F016
:103050000DFD00006C59002052656365697665645A
:103060002061206661756C74212069643A20307893
:10307000253038782C2070633A2030782530387825
:103080002C20696E666F3A20307825303878000041
:10309000024605480121008801EB004003A105F02C
:1030A000A1FA06F0E3FC00006C590020526563654C
:1030B0006976656420616E206572726F723A2030A5
:1030C00078253038782100002DE9F84F254C8146CD
:1030D000924660880E46814241D800274FF6FF781D
:1030E0008DF80070684600F0F5F822786078A188C5
:1030F000884201DA401C00E00020C0B2904204D1B6
:103100009DF8000000F032F927E065786078884289
:1031100001DA401C00E0002060709DF8000000F023
:1031200025F9454519D0A068B9F1000F40F835A040
:103130000DD066B16188E068324605FB0100494662
:10314000FEF7A2F9A06800EBC500868002E000EB64
:10315000C50087800020BDE8F88F0420FBE7092028
:10316000F9E700004458002010B50E4C03E0401C65
:1031700000E00020207020786178814210D0227811
:103180006188E068A36802FB010003EBC20153F809
:103190003220898890472078A1888842E9DAE6E7DA
:1031A00010BD00004458002030B5CB0008339DB25C
:1031B00093074FF0000401D0072030BD044B9A6004
:1031C0002A44DA605C701C7058809980002030BD01
:1031D00044580020014801F010BB00005C5800205A
:1031E00070B514460E46050004D10B4940F2C510D7
:1031F00000F000F93CB12868012EC4600AD000211B
:103200008160002070BD04494FF4E37000F0F2F8D3
:10321000072070BD0121F3E74CC20F0038B50E48FE
:1032200008235822416800910C49006802F0BEF959
:1032300000280FD10A4A69460A4801F0E3FA04005F
:1032400008D10121074801F0ACFB064901200839EB
:103250000870204638BD000028BA0F0018850020ED
:10326000EDA80F005C58002070B516460D4604000E
:1032700004D10C4940F2D51000F0BCF80A48854250
:1032800001D9072070BD0948266101F0B6FA28442B
:103290006060A06800B1A5602146BDE870400020D4
:1032A00008F030B84CC20F0017FCFF005C5800203B
:1032B00010B5040004D106494FF4F57000F09AF8F7
:1032C000002021462076BDE81040012008F01AB801
:1032D0004CC20F0070B5044607F022FA012803D053
:1032E00010A11D2000F086F8EFF3108172B61D4A80
:1032F0009368012083B990604FF0E020D0F88051AE
:10330000194B1D401560C0F88031D0F884315360EE
:103310004217C0F8842100202070002900D162B635
:1033200070BD00002E2E5C2E2E5C2E2E5C2E2E5C90
:103330002E2E5C636F6D706F6E656E74735C6C695E
:10334000627261726965735C7574696C5C617070DE
:103350005F7574696C5F706C6174666F726D2E63FB
:103360000000000070850020FC06FFBD10B504467B
:1033700007F0D6F9012803D00DA12B2000F03AF870
:103380001B498868002811D0002C0FD1EFF3108062
:1033900072B60B684FF0E022C2F800314B68C2F8F9
:1033A000043100228A60002800D162B610BD0000FE
:1033B0002E2E5C2E2E5C2E2E5C2E2E5C2E2E5C6312
:1033C0006F6D706F6E656E74735C6C696272617242
:1033D0006965735C7574696C5C6170705F75746944
:1033E0006C5F706C6174666F726D2E63000000001C
:1033F000708500201CB56A46ADF8000001910021DF
:1034000044F20200FFF716FE1CBD0000F8B51F488D
:103410000146446AC06A8D6CAC2802D1486B0544F1
:10342000241A1B4E0094042730882B4607EB0040DB
:10343000184A19A105F0E5F8224629461548FEF775
:103440005DF8E8B13088234607EB00402A4620A10A
:1034500005F0CFF804F05EFF0028FBD102F0D4FCA9
:103460002146284603F0CEFB040007D03088012116
:1034700001EB004022A100BF05F0B0F82046F8BDE6
:103480003088002407EB004024A1F5E7EC7F002002
:103490006C59002000100F00566572696679696EDC
:1034A0006720424C3A20416464723A2030782530DB
:1034B00038782C205372633A203078253038782CB5
:1034C000204C656E3A2030782530387800000000B6
:1034D000436F7079696E6720626F6F746C6F61649F
:1034E00065723A205372633A203078253038782C50
:1034F000204C656E3A203078253038780000000086
:103500005265717565737420746F20636F707920D4
:10351000424C206661696C65640000004E6F206259
:103520006F6F746C6F6164657220636F7079206E69
:1035300065656465642C20626F6F746C6F6164658F
:10354000722075706461746520636F6D706C657452
:10355000652E000030B595B0040004D12E4940F22C
:103560002740FFF747FF2D494FF6FF70224648805E
:1035700001208DF812004FF65960ADF8100004A933
:103580000120A8DF002844D1254B0FCB8DE80F0088
:10359000A11C684662DF00283BD121491C2260390A
:1035A0000BA8FDF771FF1F4D142205F1C401A86897
:1035B0001290A0788DF84A002868139006A8FDF7AD
:1035C00063FF12A8069013A807902088231D06AA5F
:1035D0000BA9AADF00281CD11C2205F1D8010BA8D9
:1035E000FDF752FFE8681290A0788DF84A006868ED
:1035F0001390142205F1F40106A8FDF745FF12A867
:10360000069013A80790208804F10C0306AA0BA9C2
:10361000AADF15B030BD0000E0BE0F000858002042
:10362000D8B90F00D0B80F00F0B585B00D46040032
:1036300004D136494FF4B370FFF7DCFE25B93349A6
:1036400040F26710FFF7D6FE14216846FDF744FFED
:103650002078032308280BD12D48C188491E89B240
:10366000C1808288002A49D0002947D1C2802370B6
:103670002178607860228DF800208DF801108DF897
:10368000020063780325012B14D0224802212278FE
:10369000008801EB004020A104F0ABFF60780B280C
:1036A00028D101F003FB8DF80300002001F006FB98
:1036B00004251FE0207809281CD2DFE800F01B1B3E
:1036C0001B211B1B051B2100D4E902706D46E91C60
:1036D000666807F05FFE044629193046C91C07F0EA
:1036E00059FE044429193846C91C07F053FE2044EA
:1036F000C01CC5B22946684607F0DAF805B0F0BD2F
:10370000D4E90112684607F0C2F8F1E7E0BE0F0005
:1037100008580020305900204446552072657175C4
:10372000657374202564206661696C65642077691F
:103730007468206572726F723A20307825780000C4
:103740002DE9F0411E4C0027217AC90734D01D49CC
:10375000884231D01C4D04261CA1288806EB00406D
:1037600004F03CFF6088A0F57F41FF3918D028881D
:103770001EA106EB004004F031FFA068132140F0C9
:103780000400A060608876DF002816D11B4CC82793
:103790004FF47A48611C404688477F1EFAD101E009
:1037A000207874DF05F07AFA070005D1288814A183
:1037B00006EB004004F012FF3846BDE8F08100003F
:1037C0000858002030CD0F00305900205368757420
:1037D00074696E6720646F776E20424C4520747266
:1037E000616E73706F72742E000000004469736321
:1037F0006F6E6E656374696E672E0000E0B80F002F
:10380000424C45207472616E73706F7274207368DD
:10381000757420646F776E2E000000002DE9F04172
:10382000204C07460020217AC90739D11E4D0426B5
:103830001EA1288806EB004004F0D0FE2348E76074
:1038400001F0D4FF00F026FB002829D103F048FC4A
:1038500038B11F4803F038FCA06840F00200A060B7
:1038600005E028881BA106EB004004F0B7FE01F03C
:10387000F1FA002814D116481C30FFF76BFE00281F
:103880000ED1FFF72FFB00280AD1A06818A140F045
:103890000100A060288806EB004004F09FFE002095
:1038A000BDE8F0810858002030590020496E697445
:1038B00069616C697A696E6720424C4520444655BF
:1038C000207472616E73706F72740000E8CD0F0027
:1038D000BC6D00204E6F20616476657274697369F7
:1038E0006E67206E616D6520666F756E6400000006
:1038F000424C4520444655207472616E73706F725D
:103900007420696E697469616C697A65642E00005F
:103910002DE9FE4FA44E0746041D018830884FF064
:103920000408A24D4FF0000A4FF00109424608EB8F
:103930000040212977D040DC132975D026DC0129ED
:1039400073D010295DD0112974D012296FD115467A
:1039500097A104F043FE3088E28805EB00409EA169
:1039600004F040FE3088A28805EB0040A0A104F0DE
:1039700039FE3088228905EB0040A3A104F032FE15
:103980003088628905EB0040A4A1EEE0142978D0CC
:103990001A2977D01F294AD1A6A104F01FFE211DA4
:1039A000688875DF040042D03188224609EB014067
:1039B000ACA104F017FE20461FE051296FD00EDCA9
:1039C00022296DD0232969D024297BD0502977D191
:1039D00003B03946BDE8F04FB04806F06BB9522944
:1039E000D7D0552939D056296AD1B879002867D15E
:1039F0001321688876DF002862D0BDE8FE4FFFF70C
:103A000047BBA7A104F0EAFD20886880E96809B1F6
:103A100001208847A549688875DF020050D03188A9
:103A200009EB014004E07FE054E086E002E047E07B
:103A30009FA19AE04FF6FF706880287A400704D46F
:103A4000FFF750FA08B1FFF723FBE968002937D0E8
:103A500003B00220BDE8F04F0847FA88F72A14D2D5
:103A60009107B1F1404F0ED0D11F8BB2591ECC1728
:103A700001EB947424F00304091B591A891D8CB2BC
:103A800004E077E07FE0144600E0F7242346944901
:103A900004F0AFFD21466888B5DFACE702E050E0F6
:103AA0003AE00FE08FA104F099FDCDF800A0CDF829
:103AB00004A0B8880022694690DF2AE0FFF7E8FA00
:103AC000BDE8FE8F6389E28803B093A1BDE8F04FA3
:103AD00004F08FBD1446A0A104F080FD734801AA34
:103AE000163842F60521806A0190CDF808D0688822
:103AF000ADDF08B1FFF7CCFA3088BDF8002004EB49
:103B000000409FA104F06EFD00231A4685216888BD
:103B10007FDF0028D2D1D3E7217900916379A279A0
:103B2000A0A104F06EFDCBE7ADA104F057FDCDF8E8
:103B300000A0208869468FDFEBE70021688866DFF8
:103B400059E7B8790028BBD03946544806F06EF8DA
:103B50000028B5D007F10801504805F013FC020019
:103B6000AED0318809EB0140A8A103B0BDE8F04F09
:103B700004F038BDB2A104F031FD00210A462088CE
:103B80000B4686DF37E7002320881A461946B1DF47
:103B900008B1FFF77DFA318803B008EB0140BDE8BA
:103BA000F04FB1A104F01ABD305900200858002090
:103BB000526563656976656420424C455F474150B4
:103BC0005F4556545F434F4E4E5F504152414D5FEB
:103BD00055504441544500006D61785F636F6E6ECF
:103BE0005F696E74657276616C3A2025640000002E
:103BF0006D696E5F636F6E6E5F696E74657276611C
:103C00006C3A202564000000736C6176655F6C611E
:103C100074656E63793A202564000000636F6E6EF0
:103C20005F7375705F74696D656F75743A20256494
:103C300000000000526563656976656420424C456A
:103C40005F4741505F4556545F434F4E4E5F504172
:103C500052414D5F5550444154455F524551554581
:103C6000535400004661696C75726520746F20754D
:103C7000706461746520636F6E6E656374696F6EE6
:103C800020706172616D6574657220726571756511
:103C900073743A203078257800000000D86D002039
:103CA000436F6E6E6563746564000000E6B80F00D4
:103CB0004661696C75726520746F207570646174FB
:103CC0006520636F6E6E656374696F6E20706172DC
:103CD000616D65746572733A203078257800000054
:103CE00098BE0F00526563656976656420424C4555
:103CF0005F4741505F4556545F444154415F4C45D6
:103D00004E4754485F5550444154455F52455155C4
:103D10004553542E00000000526563656976656462
:103D200020424C455F4741505F4556545F444154E3
:103D3000415F4C454E4754485F55504441544520DF
:103D40002825752C206D61785F72785F74696D65C8
:103D5000202575292E00000052656365697665642B
:103D600020424C455F4741505F4556545F534543A1
:103D70005F504152414D535F524551554553540098
:103D80004343434420666F722073657276696365AE
:103D9000206368616E676564206973203078253020
:103DA00034780000526563656976656420424C454D
:103DB0005F4741505F4556545F5048595F555044E6
:103DC000415445202852583A25642C2054583A250D
:103DD000642C207374617475733A256429000000A3
:103DE000526563656976656420424C455F47415082
:103DF0005F4556545F5048595F5550444154455FA4
:103E0000524551554553542E00000000436F756CC8
:103E100064206E6F742068616E646C65206F6E5FE5
:103E20006374726C5F70745F77726974652E20655D
:103E300072725F636F64653A2030782530347800A1
:103E4000526563656976656420424C455F47415021
:103E50005F4556545F5345435F494E464F5F524559
:103E6000515545535400000046696E697368656496
:103E70002068616E646C696E6720636F6E6E20737C
:103E8000656320757064617465000000007800F05F
:103E90000100704738B50020009002F0BFFE0028F6
:103EA00030D1194C0425194A208819A105EB00408E
:103EB00004F098FB154813DF002823D120881CA1AB
:103EC00005EB004004F08AFB04F012FF002819D132
:103ED000684604F063FD002814D120881AA105EB80
:103EE000004004F07BFB6946012004F061FD0028DE
:103EF00008D120881AA105EB004004F06FFB68464A
:103F000004F000FE38BD00003059002000100F0002
:103F100053657474696E6720757020766563746F7D
:103F200072207461626C653A2030782530387800F0
:103F3000456E61626C696E6720536F667444657686
:103F40006963652E00000000436F6E6669677572D5
:103F5000696E6720424C4520737461636B2E0000CC
:103F6000456E61626C696E672074686520424C45DD
:103F700020737461636B2E0011480421008801EBEB
:103F8000004010A104F02AFB04F0F6FB04F0C2F993
:103F90000028FBD1114E64254FF47A47741C384633
:103FA000A0476D1EFAD1BFF34F8F0D4801680D4A2F
:103FB00001F4E06111430160BFF34F8F00BFFDE7E3
:103FC0006C590020526573657474696E6720626F66
:103FD0006F746C6F616465722E00000060B70F0033
:103FE0000CED00E00400FA052DE9FC410646C0078F
:103FF0004FF000050ED0104F00240122385D0095CF
:1040000000231146019504F035F8641C042CF4D308
:1040100000F064F8B0070DD5074E0024361D0022CD
:10402000305D032300951146019504F023F8641CCC
:10403000042CF4D3BDE8FC8156B70F0010B504463C
:10404000042803D305A12120FFF7D4F90E4801214C
:10405000005DBDE8104004F083B800002E2E5C2EF9
:104060002E5C2E2E5C2E2E5C2E2E5C636F6D706F80
:104070006E656E74735C626F617264735C626F61B3
:104080007264732E6300000056B70F0010B504462B
:10409000042803D305A11B20FFF7ACF90E4800212B
:1040A000005DBDE8104004F05BB800002E2E5C2ED1
:1040B0002E5C2E2E5C2E2E5C2E2E5C636F6D706F30
:1040C0006E656E74735C626F617264735C626F6163
:1040D0007264732E6300000056B70F0010B5002401
:1040E0002046FFF7ABFF641C042CF9D310BD000081
:1040F0002DE9F8430546861C00208DF80000904607
:104100000F464FF001096846FFF7E4F81B4C2068A2
:104110003860D4E90001401AA168081A41F21C0174
:1041200067180EE00121384601F08BFA01F03CF9E6
:104130000146384601F085FAD4E90001401AA16829
:10414000081A401C8642EDD8B8F1000F03D00520B4
:1041500065F3891002E0062065F39F50A26821688C
:10416000114004EB8101C8602068304420609DF854
:104170000000FFF7FBF84846BDE8F8836C88002094
:1041800010B543689C18446021B905E013F8010B91
:1041900001F8010B521EF9D2012010BD30B4826823
:1041A0000468531C8360A154D0E901128A4202D3EF
:1041B00030BC03F067BC30BC70470000034803C844
:1041C000814201D101207047002070476C88002097
:1041D00010B50548012101F04AFABFF35F8F08B11D
:1041E000002010BD012010BD0058002010B5064C65
:1041F0002068012803D005A16D20FFF7FBF8BFF36D
:104200005F8F0020206010BD005800202E2E5C2EF5
:104210002E5C2E2E5C2E2E5C2E2E5C636F6D706FCE
:104220006E656E74735C6C69627261726965735CF1
:104230006D757465785C6E72665F6D74782E68005B
:1042400004490020086004494FF48060C1F88001EF
:104250007047000000A5025004E000E0034901207F
:10426000086003498002C1F80001704700A50250B0
:1042700004E000E070B500F10806106815460C4631
:10428000202802D248F2145070BDFFF7A1FF80B180
:10429000FFF7E4FF21463046FEF750FA0646FFF7E7
:1042A000CFFFFFF7A3FF304600F03EFE060003D02D
:1042B00004E048F2045070BD2020286020212046F0
:1042C00001F0EAFF304670BD10B50830FEF766FA1F
:1042D000BDE8104000F028BE2DE9F04700F10809C4
:1042E0000E461446FFF774FFB8B1FFF7B7FF4FF45F
:1042F00080584546AC4200D825462A4631460E48ED
:10430000FDF7C2F82A460C494846FEF761FA070055
:10431000A4EB05042E4404D005E048F20450BDE8A7
:10432000F087002CE5D1FFF78BFFFFF75FFF3846E2
:10433000BDE8F04700F0F8BD9C5D002070B50B486B
:1043400000240460BFF35F8F094D01202860FEF751
:104350000FFB01002C604FF0030004D0052901D1B0
:1043600048F2035070BD002070BD000000580020CE
:1043700000A50250014900200860704700A50250C6
:1043800010B5040003D10549C520FFF733F80448F0
:10439000C16B6160006CA06010BD0000E0BF0F0049
:1043A000EC7F002040684968884201D801207047AE
:1043B00000207047F0B54FF0FF3622B11268D243AB
:1043C00000230A4D0DE03246FAE7C45C624008243F
:1043D000D70700D037462F4087EA5202641EF7D134
:1043E0005B1C8B42F1D3D043F0BD00002083B8EDBD
:1043F000F0B5146906468DB020681546271DE0B15A
:10440000022920D00A2000906B4609AA304606F007
:104410000DFA00280FD009A901A8009A06F012F899
:1044200001AE96E80F0005AE86E80F0023686968C4
:104430003A4605A898470DB0F0BD0DB03046BDE82E
:10444000F04006F073B86946304606F005F80028DB
:10445000F1D0236869683A46684698470028EAD050
:1044600002980028F5D1019870600120E3E75368B5
:104470005B7813F0C00303D0402B03D000207047BB
:1044800000F002B8FFF7B4BF2DE9FF410B465168B9
:10449000064614464878334D00F00F0210F0300005
:1044A00055F8225006D0102806D0202808D03028F1
:1044B00056D13EE022694DE061690120087047E075
:1044C000022B28D1042A26D84FF00108694630462D
:1044D000676905F0C1FF00281AD009E00B7922694D
:1044E00013FB00226846A84770B13878401C38702A
:1044F000029820B1616838784A799042EED30198E9
:104500007060029860BB02E04FF00008F7E7404699
:1045100004B0BDE8F081D4E904300F79027817FBCC
:10452000023349798A421BD2521C02701A466168D2
:1045300010E008786169072A087009D1606801797C
:104540002069FCF7C9FF60682169806805F09FFF5A
:104550002269616804B03046AC46BDE8F04160476E
:104560000020D5E7ACBC0F0038B51D4901200A6812
:10457000D20301D5000407E01A490A6812F0A90F16
:1045800004D0086800F056000860002001F0B8FE72
:10459000154C0425D0B119200090684603F0B2FDF7
:1045A000D0F810050099C84010F0010F13D00D4845
:1045B000001F006810F0B10007D020880BA105EBA8
:1045C000004000BF04F00AF8012038BD208810A187
:1045D00005EB0040F6E7208816A105EB0040F1E767
:1045E00000040040200500406C590020444655203E
:1045F0006D6F64652072657175657374656420768E
:1046000069612047505245475245542E0000000032
:10461000444655206D6F64652062656361757365FE
:1046200020617070206973206E6F742076616C69F0
:10463000642E0000444655206D6F646520726571DC
:104640007565737465642076696120627574746F32
:104650006E2E0000FEB518490446086808B1401ED9
:1046600008601648D4E9015300880426227806EB36
:1046700000409DB10E6821690296CDE900312B46BC
:10468000012A16D00EA210A103F0CEFF6169002905
:1046900011D0E06803B0BDE8F04008470968009118
:1046A000012A04D006A217A103F0ABFFEEE71FA278
:1046B000F9E71EA2E7E7FEBD205800203859002088
:1046C0006572617365000000466C61736820257334
:1046D000206661696C6564202830782578293A2045
:1046E000616464723D25702C206C656E3D307825C8
:1046F000782062797465732C2070656E64696E67CA
:1047000020256400466C61736820257320737563EF
:10471000636573733A20616464723D25702C207068
:10472000656E64696E6720256400000077726974A5
:104730006500000010B508281BD2DFE800F0041265
:104740001A1A1A041A040120FFF74EFC0020FFF782
:104750009DFC0120FFF79AFCBDE810400220FFF706
:104760006DBC0120FFF76AFCBDE810400220FFF796
:104770008DBC10BD10B50446032806D0042C04D00F
:10478000062C0ED0072C04D10BE00749074801F096
:1047900069F907480168002905D02046BDE81040A6
:1047A0000847FFF7E9FB10BD19510F00C0D4010005
:1047B000B857002010B50446062802D1002002F0A8
:1047C0000FFE04480168002903D02046BDE81040D0
:1047D000084710BD0458002010B50021024800F021
:1047E00046FF80F3100010BD889800204FF4A0729F
:1047F00002EB810189B200F03BBA0068D0F80405F1
:10480000704700002DE9F04716460D46040003D11D
:1048100036492F20FEF7EEFD1DB934493020FEF752
:10482000E9FD1EB931493120FEF7E4FD60793049D8
:10483000DFF8BC80DFF8BC9041F82060617908F1B6
:10484000040808EBC100007938B10824B9F8000069
:10485000022101EB004028A143E02E882768B6F52D
:10486000805F03D32DA1FD20FEF7C4FDC7F80865C6
:10487000AD7894F90460A81E022806D3681F0328A7
:1048800003D331A14520FEF7B5FD002E4FEA4510B8
:1048900006DA06F00F0101F1E02181F8140D03E0C2
:1048A00006F1E02686F8000494F90410012201F0D4
:1048B0001F0302FA03F04909890001F1E021C1F860
:1048C0008002C1F80001617908EBC1010A716179C8
:1048D00048F83140B9F80000032101EB0040002402
:1048E00024A103F07BFE2046BDE8F08790C20F00B4
:1048F0007C5800205059002052544320696E737434
:10490000616E636520616C726561647920696E69AE
:104910007469616C697A65642E0000002E2E5C2E2D
:104920002E5C2E2E5C2E2E5C2E2E5C6D6F64756CB4
:1049300065735C6E7266785C68616C2F6E72665F20
:104940007274632E680000002E2E5C2E2E5C2E2EBC
:104950005C2E2E5C2E2E5C696E74656772617469C4
:104960006F6E5C6E7266785C6E7266785F676C758F
:10497000652E68005254433A20696E697469616C0F
:10498000697A65642E00000090F90400012100F0AE
:104990001F0291404009800000F1E020C0F80012A1
:1049A00070470A46022100F04FB94FF4827100F0BF
:1049B0005FB9000010B5040003D104496120FEF77F
:1049C00019FD20680121016010BD000090C20F0098
:1049D00010B5040003D104496720FEF70BFD2068E1
:1049E0000121416010BD000090C20F002DE9F84385
:1049F000994616460F46050003D12B498620FEF73F
:104A0000F9FC29684FF480344FF4A070BC4000EBEF
:104A1000870080B226F07F46C1F808432968C1F8B4
:104A20004843296800220A5008580090286800EB83
:104A30008701D1F84005C1F840652968D1F804150F
:104A40001A4F401A20F07F404FF00408012809D186
:104A5000398808EB014016A103F0C0FD21494FF44D
:104A6000046088472868C0F844432968D1F80435B1
:104A7000F01A20F07F40020201D540F07F40C9F1DA
:104A8000000290420BDD022809DC3988324608EB2F
:104A9000014015A103F0ADFD0D20BDE8F883C1F87C
:104AA00004430020F9E7000090C20F005059002095
:104AB0005254433A2044656C617920696E74726F78
:104AC00064756365642064756520746F2072697312
:104AD0006B206F66207072652D666972696E672E35
:104AE0000000000041BA0F005254433A2057696E4B
:104AF000646F77656420636F6D70617265207365A4
:104B0000742074696D656F757420286162735F76B7
:104B1000616C75653A25642C20636F756E746572DF
:104B20003A2564292E0000002DE9FC4180461F46ED
:104B300015460E4600240D4800F080FD38B11120C6
:104B4000BDE8FC8106EB043003F0EEFE641CAC42D1
:104B5000F8D1064800F069FDCDE900573346002240
:104B60000221404600F02AF80020E9E7885800209A
:104B70002DE9F843104D0F4680461E469146694682
:104B8000286800F026FD040014D01C21FCF7A4FCCA
:104B900001202071C4F81490380BC4F80080C4E9D7
:104BA00002606946286800F035FD05F01FFE002010
:104BB000BDE8F8830420FBE784BA0F002DE9F04339
:104BC00087B00446DDE90E8980681D4616460F460B
:104BD00000280BD018216846FCF77EFC02A88DF84F
:104BE000007080E86003A1686846884707B0BDE8A8
:104BF000F08330B50446006887B00D468068002811
:104C00001FD018216846FCF767FC0195A068059045
:104C1000207910B1012810D107E001208DF80000A3
:104C200020690290E068039005E002208DF8000002
:104C3000E06800030290606904902068816868461B
:104C4000884707B030BD000070B516460C46050019
:104C500003D10649B920FEF7CDFB2868C0F84443CC
:104C6000002E02D02868C0F8044370BD90C20F0027
:104C700038B50C46050003D10749CA20FEF7BAFB38
:104C80002868015929B100210151005900900120E3
:104C900038BD002038BD000090C20F000B2803D3A0
:104CA0000B38C0B200F00AB8704700000249002279
:104CB00008780A70704700002458002001490870E5
:104CC0000B207047245800200149012008707047CC
:104CD000F95700202DE9FE4307004FF020009046D1
:104CE00089464FF00106029004D12A494FF4FA7028
:104CF000FEF780FB284C0425434620884A4605EBF6
:104D0000004026A103F075FC02A93348CDE900015B
:104D100043464A463149A0F59A7001F0CDF90200A8
:104D200007D02088012101EB00402DA103F05AFC9F
:104D30002CE007F16F0120220F462748FCF7DEFB2D
:104D400028B32088022101EB004032A103F046FC89
:104D5000208837A105EB004003F040FC208820228A
:104D600005EB0040394603F0E5FB208835A105EB53
:104D7000004003F033FC2088202205EB0040164958
:104D800003F0D8FB03F0C6FA0028FBD1002630461A
:104D9000BDE8FE83B8C10F00485900204861736820
:104DA00020766572696669636174696F6E2E20464C
:104DB00069726D77617265207374617274206164C9
:104DC00064726573733A20307825782C2073697A81
:104DD000653A203078257800F88400209CB70F00D1
:104DE000436F756C64206E6F742072756E206861FD
:104DF000736820766572696669636174696F6E2095
:104E0000286572725F636F64652030782578292E7B
:104E10000000000048617368207665726966696306
:104E20006174696F6E206661696C65642E000000B4
:104E300045787065637465642046572068617368BF
:104E40003A00000041637475616C20465720686128
:104E500073683A003EB59DF8080020F00F00401C32
:104E600020F0F00010308DF8080068466DDF002853
:104E70002AD19DF80100401C8DF8010068466CDFC6
:104E8000002821D111481249007A82074FF004000E
:104E90000BD5104C0988221D00EB01400EA1A3691F
:104EA00003F0A7FB211DA06907E0098800EB014082
:104EB00012A103F093FB19A1072082B202A87CDFA4
:104EC000002801D117487ADF3EBD000008580020B5
:104ED00030590020BC6D002053657474696E6720E2
:104EE000616476206E616D653A2025732C206C65B7
:104EF0006E6774683A202564000000005573696E7F
:104F0000672064656661756C74206164766572748F
:104F10006973696E67206E616D6500004466755443
:104F200065737400E6B80F0010B50F4C48F20351DA
:104F3000031B48F21652A04211D007DC00280AD009
:104F40000A4BC01808D0012804D10BE00A2B01D06D
:104F50000D2B07D0104610BD48F2015010BD48F28D
:104F6000025010BD084610BD0202F00000FE0FFF07
:104F70002DE9FC5F0646DFF804A1984615460F466A
:104F80004FF0040BB1420BD1BAF8000033460BEBE3
:104F900000403A463AA103F02CFB0020BDE8FC9FFC
:104FA00004D243494FF02900FEF724FAB8F1000F6C
:104FB00003D13F492A20FEF71DFA300503D03C49B2
:104FC0002B20FEF717FAB81B040B03D138492E200B
:104FD000FEF710FA0020009005F6FF704FEA103936
:104FE00000F024FF4046A04500D20446A04641E020
:104FF0004946C14504D808462C46CDF8049004E043
:1050000040464FEA0834CDF804800146002230467D
:1050100001F096FC0028C1D10094BAF80010334684
:105020000BEB01403A4623A103F0EBFA601E00F0BF
:105030000300221A002339463046D21C01F030FD0D
:105040000028ABD101992448A9EB01092D1B016B64
:105050002644214401632744002002F00BF900900C
:1050600040B1BAF80000012101EB00401BA103F0A0
:10507000B5FA01E0002DBBD100988FE76C590020F4
:105080004E6F20636F7079206E6565646564207370
:1050900072635F616464723A20307825782C2064F2
:1050A00073745F616464723A203078257800000080
:1050B000A4BD0F00436F7079696E67203078257842
:1050C00020746F20307825782C2073697A653A2017
:1050D0003078257800000000EC7F00204661696C84
:1050E000656420746F20777269746520696D6167EB
:1050F0006520636F7079696E672070726F67726583
:10510000737320746F2073657474696E6773207095
:105110006167652E0000000004480321008801EB50
:10512000004003A103F05AFAFEF726FF6C59002055
:10513000496E61637469766974792074696D656F0D
:1051400075742E00014941600020704758BA0F0065
:1051500010B50B4941600B4800F070FA68B903F0D4
:1051600019FE08491C234FF4EE7208740448A1F597
:10517000EE71001F006800F019FA002010BD000059
:1051800088BA0F00588700202DE9FC5F0E00834687
:10519000DDE90C47C6F1000098469246814600D4EE
:1051A0000846012503E000BF90FBFAF06D1C504556
:1051B000FADAA84500D9454624B1002E01DB78076C
:1051C00000D5641EB80702D5B8F1000F0AD0F80761
:1051D00008D13CB1A54205D220215846641EFEF7F5
:1051E000DDFFF6E7002E02DA4E462D2102E07807B9
:1051F00003D52B215846FEF7D1FF07F00300022804
:105200000BD1B8F1000F08D13CB1A54205D2302135
:105210005846641EFEF7C2FFF6E7CDE90047434655
:1052200052463146584606F0D7F8BDE8FC9F0000CC
:1052300010B5024600201268930702D0530702D42B
:1052400010BD500719D502F00300012807D002282D
:105250000BD00D494FF49170FEF7CCF80BE0C2F380
:1052600083100B68801C184404E00223086803EBD9
:10527000925210440860012010BD086800EB925360
:10528000C2F38910401CEEE7B0C70F000248006867
:10529000002800D001207047885800200248007A7A
:1052A000002800D0012070475887002038B54FF4FF
:1052B00040531A4A5D6800F50051954204D0486891
:1052C000904201D1012400E00024954224D1486895
:1052D000904221D11878142801D95A6900E000229F
:1052E0000F48B2FBF0F30A78142A01D9496900E0AB
:1052F0000021B1FBF0F0834203D0012409A2009009
:1053000002E0002409A200900A480321008801EB72
:10531000004009A103F075F9204638BDDBE5B15125
:1053200040420F006D616A6F720000006D696E6F20
:105330007200000048590020536F66744465766916
:105340006365207570646174652069732061202530
:10535000732076657273696F6E2075706461746511
:105360002E2043757272656E743A2025642E204E8D
:1053700065773A2025642E0070B5054608680C460E
:105380004A6886682846314604F0A2FF60682861B2
:1053900004F10C00686170780221B1EB901F01D11B
:1053A000241D2C6170BD00002DE9FF410026264818
:1053B00000F041F92448001F074600F03CF9234C57
:1053C00060680090A56800E000986946284004EBFA
:1053D00080000C30FFF72CFF0028F5D101AA0099BE
:1053E00001EA050304EB8303491CDB6842F8203023
:1053F000401C00910228F2D3019800F0030001281C
:105400001AD002280ED012494FF4AF70FDF7F2FF08
:10541000384600F00DF908B10098606004B03046DD
:10542000BDE8F0810198032101EB90500099BDF88F
:105430000A6001EB900005E00198BDF80A60C0F336
:10544000831008440090E3E7849800206C880020D3
:10545000B0C70F0070B500224FF48051104600F025
:1054600009FBC8B912480022C0F57E2100F002FBFA
:1054700090B94FF400410F4803F03AF902F034FFBD
:105480000D4C03250DA1208805EB004003F0A6F884
:105490000D4800F00BFC08B1FDF7FAFD00F0FAF939
:1054A00020880AA105EB004003F098F8002070BDA9
:1054B00000100F00D5310F006C590020496E736940
:1054C0006465206D61696E0035470F004166746543
:1054D00072206D61696E00002DE9F05FC7888A4611
:1054E000191D1646B1FBF7F2B1FBF7F507FB1219D0
:1054F00099193944C91CB1FBF7F104464079C9B286
:10550000DDF828B0884206D217499420FDF772FFD3
:1055100001E024686D1E002DFBD1A846A7EB09050C
:10552000B5421AD81CE000BFBBF1000F06D004EB57
:1055300009010AEB08002A46091D05E004EB0900F1
:105540000AEB08012A46001DFBF79EFF2468761B24
:105550004FF00009A844B74201D9354600E03D4666
:10556000002EE1D1BDE8F09FD4C20F0030B5024655
:1055700059B103F0E9F80021074C09E004EB81037D
:1055800015685B88AB4202D11160002030BD491C18
:105590008142F3D3052030BD2459002010B5FBF71C
:1055A00088FE08B1002010BD112010BD10B531B12A
:1055B000B2FBF3F403FB14241CB1092010BD0E2030
:1055C00010BD01600021416081608281C381084675
:1055D00010BD70B50C460546FBF720FE002802D032
:1055E00021882868084470BD10B50A8849888A4215
:1055F00003D1FBF755FE012010BD002010BD70B592
:105600000C460546FBF72FFE002802D0618828686B
:10561000084470BD10B50A8849888A4203D1FBF757
:1056200019FE012010BD002010BD002100F00FB8B0
:10563000002100F012B8012100F01EB8012100F095
:1056400011B808B56A46FBF780FE009808BD08B59A
:105650006A46FBF760FE009808BD08B56A46FBF78E
:105660005AFE08BD08B56A46FBF748FE08BD08B5F6
:105670006A46FBF737FE08BD08B56A46FBF73EFEF3
:10568000009808BD08B56A46FBF76CFE009808BD97
:1056900038B5040003D115A1FE20FDF7ABFE0025AF
:1056A0008DF800506846FDF715FE206862680168B5
:1056B000914214D9491E01600D781CB919A1C2206C
:1056C000FDF798FEA08AE16805FB00152068217AA5
:1056D0000278891A0279C9B28A4200D201719DF812
:1056E0000000FDF743FE284638BD00002E2E5C2E3C
:1056F0002E5C2E2E5C2E2E5C2E2E5C636F6D706FDA
:105700006E656E74735C6C69627261726965735CFC
:1057100062616C6C6F635C6E72665F62616C6C6F11
:10572000632E63002E2E5C2E2E5C2E2E5C2E2E5CA5
:105730002E2E5C636F6D706F6E656E74735C6C693A
:10574000627261726965735C62616C6C6F635C6EDE
:1057500072665F62616C6C6F632E630038B50C46D5
:10576000050004D112A140F22110FDF743FE24B937
:105770000FA14FF49170FDF73DFE00208DF8000061
:105780006846FDF7A7FD1DB91749CF20FDF732FE8A
:10579000E8682A68211AA88AB1FBF0F11068431C56
:1057A000136001709DF80000FDF7E0FD38BD0000BA
:1057B0002E2E5C2E2E5C2E2E5C2E2E5C2E2E5C63EE
:1057C0006F6D706F6E656E74735C6C69627261721E
:1057D0006965735C62616C6C6F635C6E72665F625C
:1057E000616C6C6F632E630024570F0010B50400CA
:1057F00002D0206830B901E00E2010BD17A1D920D9
:10580000FDF7F8FD606818B914A1DA20FDF7F2FD84
:10581000A06818B911A1DB20FDF7ECFDE06818B90C
:105820000EA1DC20FDF7E6FDA08A18B90BA1DD2052
:10583000FDF7E0FD207A61682268401AC0B211606D
:1058400004E0226811684B1C13600870401EC0B24F
:10585000F7D221680020087110BD00002E2E5C2EAA
:105860002E5C2E2E5C2E2E5C2E2E5C636F6D706F68
:105870006E656E74735C6C69627261726965735C8B
:1058800062616C6C6F635C6E72665F62616C6C6FA0
:10589000632E63002DE9F041184D4FF48052042728
:1058A0002888164607EB004015A102F09BFE4FF03A
:1058B000E024D4F8802128881FA107EB004004F5DC
:1058C000C07402F08FFE60172060C4F800016060B1
:1058D000C4F8040101F0AEF930B12888012101EBD0
:1058E000004020A102F07AFE02F014FD0028FBD156
:1058F0003046BDE8F04100F051B800006C5900207E
:1059000052756E6E696E67206E72665F626F6F743D
:105910006C6F616465725F6170705F7374617274E3
:10592000207769746820616464726573733A20300B
:10593000782530387800000044697361626C696EC4
:105940006720696E74657272757074732E204E567E
:1059500049432D3E494345525B305D3A203078251E
:10596000780000004661696C65642072756E6E692E
:105970006E67206E72665F6466755F6D62725F69E6
:1059800072715F666F72776172645F616464726581
:1059900073735F73657428290000000070B50646B4
:1059A0001F4888B0C0F57F21002200F063F8021E76
:1059B0004FF0FF3507D01B480121008801EB004064
:1059C00019A102F00FFEEFF30580D6E90046C005ED
:1059D000C00D4FF0000181F3148881F3108881F32A
:1059E000118881F3138813D020221D496846FBF7E4
:1059F0004BFD203C2022694620460696FBF744FDDD
:105A00006FF0060229462046FBF704FC08B070BD83
:105A100008B0324629462046BDE87040FBF7FABB85
:105A200000100F006C590020436F756C64206E6F7E
:105A3000742070726F7465637420626F6F746C6F22
:105A40006164657220616E642073657474696E6749
:105A5000732070616765732C20307825782E0000E4
:105A600068B70F000A4601460148006805F066BCA9
:105A700088B70F0070B50B0502D1B0F57F2F01D9A3
:105A8000072070BD0AB1062500E00225104A114B1F
:105A90001468082C01D3042070BD03EB0416C6F86B
:105AA0000008C6F80418C6F80858641C146003EB14
:105AB0000414D4F8F0678642EAD1D4F8F4678E4231
:105AC000E6D1D4F8F847AC42E2D1002070BD000026
:105AD000BC57002000E001402DE9F0473D4C042573
:105AE0003B4E2088002705EB00403BA102F076FDED
:105AF000B06801280FD0A52816D0AA281DD0AC2840
:105B0000208824D0032101EB00403CA102F066FD77
:105B10000020BDE8F08720883FA105EB004002F09F
:105B20005DFDFDF70BFA10E020883EA105EB00407B
:105B300002F054FD04F062FF10E020883CA105EB68
:105B4000004002F04BFDFDF761FC024608E005EB6A
:105B500000403AA102F042FD05F020F8024601277C
:105B60004FF0010932B12188B36809EB014037A138
:105B700002F03FFD304600F055FCDFF804810021C3
:105B800088F800103F4801F075FB064698F80000C1
:105B900020B93D4940F27910FDF72CFC46B121882F
:105BA00009EB014039A102F019FD03263046B0E7A8
:105BB0000126002FFAD0012000F0A2FB0028F5D02A
:105BC0002088394905EB004002F008FD0226EDE788
:105BD000108000206C590020456E746572206E7232
:105BE000665F626F6F746C6F616465725F66775F2A
:105BF0006163746976617465000000004E6F206611
:105C000069726D7761726520746F20616374697663
:105C10006174652E0000000056616C69642041705B
:105C20007000000056616C6964205344000000005D
:105C300056616C696420424C0000000056616C693A
:105C400064205344202B20424C00000041637469BF
:105C5000766174696F6E206661696C65642077692E
:105C60007468206572726F72202564202862616EEC
:105C70006B20636F64653A20307825782900000036
:105C8000F9570020C94C0F00A4BD0F00436F756C7D
:105C900064206E6F74207772697465207365747404
:105CA000696E67732E0000003CBE0F00F8B5354CDE
:105CB00005460426208834A106EB004002F08EFC45
:105CC0003748056019200090684602F01BFA009AD8
:105CD000344900EB8200C0F80017002001F034FACC
:105CE000002842D1FFF7F8FE20B1012820D0022879
:105CF0003BD104E02C4DFEF737FC10B932E042F204
:105D0000107500F093F8294A20211820FDF74CFA6D
:105D100008B1FDF7BDF92648016811F0B10F03D0B5
:105D2000016801F04E01016000F050FFE8B901E0A8
:105D3000FEF722F91F492846FFF794FE1E4800F09F
:105D4000FDFE90B920881DA106EB004002F046FC44
:105D500000F05AF8FDF708FA02F0DCFA0028F7D153
:105D600041DFF5E701F078F908B10320F8BDFFF74E
:105D700091FD2088012101EB004014A102F02EFCCE
:105D8000F3E700006C590020496E206E72665F6276
:105D90006F6F746C6F616465725F696E6974000027
:105DA000B85700200C000300C0D401007C5900202B
:105DB0001C05004019510F0075470F00456E7465B2
:105DC00072206D61696E206C6F6F700053686F7523
:105DD0006C64206E6576657220636F6D6520686502
:105DE00072653A204166746572206E72665F626FFA
:105DF0006F746C6F616465725F6170705F73746102
:105E0000727428290000000010B503F0CBF90028B7
:105E100003D0BDE8104005F0F1BB10BD0A460146B5
:105E20000148406805F08ABA88B70F002DE9F041B3
:105E3000224C207800283FD103F0B4F9204E0327EC
:105E40004FF0010800282FD01E4800681EA1450908
:105E500030882A4607EB004002F0C4FB05EB450002
:105E6000850842F21070854201D2012000E0002036
:105E7000607005F0C3FB607820B9124808300068F4
:105E8000C0070AD030882A4607EB004014A102F070
:105E9000A9FB1F492846FFF7C1FF4FF0E0214FF44F
:105EA0008030C1F8000105E030881AA107EB0040FE
:105EB00002F094FB84F80080BDE8F081FA570020DE
:105EC0002C5900200405014057445420656E61623E
:105ED0006C6564204352563A2564206D73000000BF
:105EE0005374617274696E6720612074696D6572A4
:105EF00020282564206D732920666F7220666565F1
:105F000064696E67207761746368646F672E000050
:105F100039B60F00574454206973206E6F742065A2
:105F20006E61626C6564000070B504460D46202207
:105F3000083000F077F9202205F1200104F1280053
:105F400000F070F9002070BDF0B599B00D46214900
:105F50001E9E944607460160202B00D320231C463A
:105F60001A46614611A800F05DF92022314601A8C9
:105F700000F026F918480121FFF779FBBFF35F8F86
:105F8000002618B148F2045019B0F0BDFEF766F9CA
:105F900011AB01AA05F1080138460094FCF7BAFBE1
:105FA0000446FEF74DF90C4D2868012803D00BA1DB
:105FB0006D20FDF71FFABFF35F8F2E6044B11448C8
:105FC000C44202D148F24250DEE748F21650DBE705
:105FD0000020D9E7DD55AABB005800202E2E5C2EEC
:105FE0002E5C2E2E5C2E2E5C2E2E5C636F6D706FE1
:105FF0006E656E74735C6C69627261726965735C04
:106000006D757465785C6E72665F6D74782E68006D
:106010007CF70FFF70B516460C46054600F0E9F810
:1060200000280ED1AA791946304600F0EFF8002872
:1060300007D131462046FFF777FF002801D10149FB
:10604000216070BD7052464D2DE9F84F6C460E46EA
:10605000D4E90A7905469A4690461649304600F03A
:10606000BCF80028A54611D1706849464079420025
:10607000384600F0CBF80028A54607D1B8F100005B
:1060800001D02DB107E0A54648F21050BDE8F88FC9
:10609000AAB06D464DB182B00246534631462846FD
:1060A0000097FFF751FFA546F0E748F21550A546C7
:1060B000ECE700007052464D2DE9F0411D46DDE948
:1060C00006871646044600F02DF800280DD12A4612
:1060D0003146204600F03CF8002806D13A464146B9
:1060E0002046BDE8F04100F002B8BDE8F08170B58F
:1060F00015460E46044605F071FA002807D13EB158
:1061000060682968C268914205D248F2145070BD97
:1061100048F2135070BD83682A4631462046BDE8D8
:106120007040184710B550B161B14160096804462C
:106130008847002802D105482060002010BD48F2A1
:10614000015010BD48F2105010BD00006E5246487C
:1061500070B515460E46044605F040FA00280BD1EE
:1061600046B155B160682A46314643682046BDE8CD
:106170007040184748F2105070BD002070BD0000FC
:106180002DE9F0410B480C4D0C4F401BC608012077
:106190003870002406E000BF55F83400804700281E
:1061A00005D1641CB442F7D3022038700020BDE84A
:1061B000F081000030CD0F0028CD0F00FC570020EB
:1061C00070B514460D46064600F02CF82919301912
:1061D0002246BDE8704000F025B828B1006888422A
:1061E00005D048F24050704748F2105070470020E8
:1061F000704728B139B10022C1E90020104670472C
:1062000048F21050704748F21350704720B1914245
:1062100005D048F21150704748F2105070470020E6
:106220007047000070B516460C46050003D10AA160
:106230001F20FDF7DFF81CB907A12020FDF7DAF8D1
:10624000A919491E04E000BF14F8010B01F8010967
:10625000A942F9D270BD00002E2E5C2E2E5C2E2E8F
:106260005C2E2E5C2E2E5C636F6D706F6E656E748F
:10627000735C6C69627261726965735C6372797078
:10628000746F5C6E72665F63727970746F5F73684F
:10629000617265642E63000070B50D46040003D181
:1062A00007A10D20FDF7A6F86019401E05E0217832
:1062B000027804F8012B00F80119A042F7D270BD52
:1062C0002E2E5C2E2E5C2E2E5C2E2E5C2E2E5C63D3
:1062D0006F6D706F6E656E74735C6C696272617203
:1062E0006965735C63727970746F5C6E72665F630C
:1062F000727970746F5F7368617265642E630000F9
:106300002DE9F041174C07460425208816A105EB1E
:10631000004002F063F91B4E306A012804D0208847
:1063200019A105EB00400FE09FB1F06988B100F0C2
:1063300055F80022B169FEF73DF8F169814208D0B5
:10634000208819A105EB004002F048F90020BDE8C3
:10635000F081208819A105EB004002F03FF90120EF
:10636000F5E700006C590020456E746572206E726E
:10637000665F6466755F6170705F69735F76616C9C
:1063800069640000EC7F002052657475726E2066AF
:10639000616C736520696E2076616C696420617040
:1063A0007020636865636B0052657475726E206659
:1063B000616C736520696E204352430052657475A9
:1063C000726E20747275652E204170702077617333
:1063D0002076616C69640000AFF300804FF4405098
:1063E000074A4168914207D18068411EC1F30B0101
:1063F000401A00F6FF7070474FF48050704700005D
:10640000DBE5B15100B5FFF7E9FF054989690A18D5
:10641000401E0844C0F30B00101A00F6FF7000BDC8
:10642000EC7F002000210160416081600148016330
:1064300070470000EC7F00202DE9FF5F7E4C0425B3
:106440007EA1208805EB004002F0C8F8208883A1D7
:1064500005EB0040009A02F0C5F8019808B185A24A
:1064600000E086A2208887A105EB004002F0BAF880
:10647000029808B17FA200E080A2208886A105EBE7
:10648000004002F0AFF8039808B17AA200E07BA2C6
:10649000208885A105EB004002F0A4F84FF440509D
:1064A00041688748814201D172A200E073A220882E
:1064B00084A105EB004002F095F8208885A105EB4A
:1064C000004002F08BF8874E208887A105EB004042
:1064D000B369326A02F08DF820888BA105EB004089
:1064E000736AF26A02F085F84FF00008DFF838B2FC
:1064F000A146AA461AE00127C0B1012820D0B8F170
:10650000020F2CD08949A420FCF774FF00255D45BB
:1065100003D98649A920FCF76DFF85480099401BE7
:10652000A0F5405088421DD201261CE0FFF76AFF0B
:106530000546029888B16B48006A01280BD00CE030
:10654000FFF74CFF0546039828B94FF440504168C7
:106550005B48814201D00127D9E70027D7E74FF4F4
:106560008055D4E700260198B9F8001046EA0004E7
:106570000AEB014042466FA102F034F8B9F800106E
:106580002A460AEB01406EA102F02CF80EB139A2A6
:1065900000E03AA2B9F800104D460AEB01406EA1A6
:1065A00002F020F80FB133A200E034A22888A946F7
:1065B00055460AEB00406EA102F014F80CB12DA272
:1065C00000E02EA2B9F800006EA105EB004002F039
:1065D00009F8BC4308D0B8F1020F05D208F1010058
:1065E000C0B28046022886D95EB1B9F80000022107
:1065F00001EB004068A101F0F1FF042004B0BDE808
:10660000F09FB8F1000F0AD0B9F800100AEB014072
:106610006CA101F0E3FF33481830FFF703FF314A64
:10662000002010610120506102F12400FFF7FAFE02
:10663000009850620020E1E76C590020456E7465B7
:1066400072206E72665F6466755F63616368655F22
:10665000707265706172652829000000726571753D
:10666000697265645F73697A653A20307825782E9F
:1066700000000000747275650000000066616C73B4
:106680006500000073696E676C655F62616E6B3AEE
:106690002025732E000000006B6565705F617070CF
:1066A0003A2025732E0000006B6565705F736F667E
:1066B000746465766963653A2025732E00000000D6
:1066C000DBE5B15153445F50524553454E543A2097
:1066D00025732E0042616E6B20636F6E74656E745D
:1066E000733A0000EC7F002042616E6B2030206323
:1066F0006F64653A203078253032783A2053697AD1
:10670000653A20307825780042616E6B2031206335
:106710006F64653A203078253032783A2053697AB0
:10672000653A20307825780000E00E002CC00F007C
:1067300000100F00706173733A2025642E00000072
:1067400063616368655F616464726573733A203086
:106750007825782E0000000063616368655F746FC0
:106760006F5F736D616C6C3A2025732E0000000022
:106770006B6565705F6669726D776172653A202539
:10678000732E000064656C6574655F6D6F72653AA9
:106790002025732E0000000041626F7274696E67DD
:1067A0002E2043616E6E6F7420666974206E65776B
:1067B000206669726D77617265206F6E2064657600
:1067C00069636500496E76616C69646174696E67BE
:1067D000206170702E00000070B50C46050004D1D9
:1067E000224940F22D10FCF705FE24B91F494FF451
:1067F0009770FCF7FFFD2A7804201D49092A2DD245
:10680000DFE802F02C052C0B182C1E2C1200214660
:106810002846BDE8704002F0CDBC098800EB01407D
:1068200014A101F0DBFE14E021462846BDE87040CB
:1068300002F05ABD21462846BDE8704002F0F6BC81
:10684000098800EB014014A101F0C8FE4FF48070EC
:10685000E0602046BDE87040FDF792BDBDE87040A5
:10686000024940F24D10FCF7C5BD0000E0BF0F002B
:106870003C59002048616E646C65204E52465F446E
:1068800046555F4F505F4352435F4745542028634E
:106890006F6D6D616E64290048616E646C65204E99
:1068A00052465F4446555F4F505F4F424A454354FE
:1068B0005F53454C4543542028636F6D6D616E6492
:1068C0002900000070B50E46040004D11B4940F2B7
:1068D0004620FCF78FFD26B9184940F24720FCF707
:1068E00089FD20780125092820D2DFE800F01F0566
:1068F0001F0F141F1A1F0A003146204602F0C6FD62
:1069000019E03146204603F00BF814E031462046EA
:1069100002F080FD0FE03146204602F0CBFE054636
:1069200009E03146204602F0B3FF04E003494FF48A
:106930001A70FCF75FFD284670BD0000E0BF0F0035
:106940002DE9F843134C0746134E20680D4600907E
:1069500030880421904601EB00402B463A460FA1B7
:1069600001F04FFE43462A4639461C4801F0DEF945
:1069700005000AD03088022101EB00402A4618A108
:1069800001F030FE2846BDE8F8832068401C2060F6
:10699000F8E7000020580020385900206E72665F2A
:1069A0006673746F726167655F6572617365286194
:1069B0006464723D307825702C206C656E3D2564D2
:1069C000207061676573292C207175657565207568
:1069D000736167653A2025640000000010590020AB
:1069E0006E72665F6673746F726167655F65726110
:1069F00073652829206661696C656420776974680D
:106A0000206572726F7220307825782E00000000A9
:106A10000B4910B504220988002802EB01421046F8
:106A200004D008A101F0DAFD104903E010A101F043
:106A3000D5FD1949BDE810400022184801F0D6B92B
:106A400038590020496E697469616C697A696E67AA
:106A5000206E72665F6673746F726167655F7364E0
:106A6000206261636B656E642E00000094BA0F00B3
:106A7000496E697469616C697A696E67206E7266C5
:106A80005F6673746F726167655F6E766D632062B7
:106A900061636B656E642E0064BA0F0010590020AC
:106AA0002DE9FC47154C8046154E20680F46CDE970
:106AB0000020308804219946154601EB00403B46F2
:106AC0004246104901F0A6FD2B463A4641460E4883
:106AD000CDF8009001F052FA05000AD0308802216A
:106AE00001EB00402A4609A101F07CFD2846BDE8E3
:106AF000FC872068401C2060F8E700002058002038
:106B00003859002028BF0F00105900206E72665FB0
:106B10006673746F726167655F777269746528293F
:106B2000206661696C65642077697468206572729B
:106B30006F7220307825782E0000000070B5104963
:106B4000104D08602888032101EB00400EA101F0E0
:106B500045FD0020FDF72EFE104800F09FFC0400CC
:106B600009D02888012101EB004022460CA101F048
:106B700039FD204670BDBDE87040084800F0C8B837
:106B8000045800206C590020456E746572696E6768
:106B900020444655206D6F64652E0000B5470F00F8
:106BA000436F756C64206E6F7420696E6974616CDC
:106BB000697A6520444655207472616E73706F72F5
:106BC000743A20307825303878000000054810B538
:106BD0000088042101EB004003A101F0FFFC00202C
:106BE00010BD00006C590020696E207765616B2034
:106BF0006E72665F6466755F696E69745F757365F2
:106C0000720000001FB58908002201AB009283E8E2
:106C10000700684618DF04B010BD00001FB5044B24
:106C20000FCB8DE80F00684618DF04B010BD0000E0
:106C3000E8B90F0070B50A4C04254FF4805620883F
:106C400008A105EB004001F0C9FCE8060BA10660B5
:106C50002088002605EB004001F0C0FC304670BDE6
:106C60006C59002072756E6E696E672069727120B2
:106C70007461626C65207365740000004166746520
:106C8000722072756E6E696E672069727120746110
:106C9000626C65207365740070B50E460178124C05
:106CA000062901D0012901D1017C2170217801251B
:106CB00001290FD0022911D00C480121008801EBD5
:106CC00000400BA101F08AFC0020207005207070AC
:106CD000284670BD3146FFF77FFDF9E73146FFF7E3
:106CE000F1FD0546F4E70000285800203C5900203B
:106CF000496E76616C6964206F626A6563742074A2
:106D000079706520696E20726571756573742E00E7
:106D100010B5040011D00120FFF77AFE00280BD136
:106D200000F016FC00F02CFD48B10949081F00F0E6
:106D30009DFC012803D0032010BD072010BD04488E
:106D40000838C4600020FDF7B9FF002010BD000026
:106D50003058002010B5816879B1094A1821FCF734
:106D6000B3F9040007D007480221008801EB004076
:106D700005A101F033FC204610BD072010BD000026
:106D8000A56D0F003C5900205363686564756C6500
:106D9000722072616E206F7574206F66207370614F
:106DA00063652100AFF30080F0B50446806887B0CA
:106DB00020B946494FF42870FCF71CFB18224449BF
:106DC0006846FAF761FB20788DF8000022780426E7
:106DD000404F414D0D2A5AD2DFE802F00752375298
:106DE0005259523E522D0F28480028883BA106EBED
:106DF000004001F0F3FB012024E0288840A106EBCD
:106E0000004001F0EBFB4FF08050D0F800110191F1
:106E1000D0F804110291D0F80C1189020491D0F835
:106E2000101189020391006905903AE069462046F5
:106E300002F064FE35E028883AA106EB004001F03C
:106E4000CDFB207C8DF804002BE028883BA106EBCD
:106E5000004001F0C3FB24E0288841A106EB00407C
:106E600001F0BCFB208AADF804001AE0288843A199
:106E700006EB004001F0B2FBF9680720884710E0FC
:106E800069462046FFF708FF58B907B0F0BD2888CB
:106E9000032101EB00403FA101F0A4FB02208DF88B
:106EA000010028889DF8012006EB004041A101F077
:106EB00099FBD4E90112684690479DF8010001282A
:106EC000E3D0F96805208847DFE70000E0BF0F0046
:106ED00010BA0F00285800203C59002048616E6409
:106EE0006C65204E52465F4446555F4F505F50528E
:106EF0004F544F434F4C5F56455253494F4E00003D
:106F000048616E646C65204E52465F4446555F4F43
:106F1000505F48415244574152455F56455253498C
:106F20004F4E000048616E646C65204E52465F44CF
:106F300046555F4F505F50494E47000048616E64B0
:106F40006C65204E52465F4446555F4F505F524538
:106F500043454950545F4E4F5449465F5345540092
:106F600048616E646C65204E52465F4446555F4FE3
:106F7000505F4D54555F47455400000048616E64B2
:106F80006C65204E52465F4446555F4F505F41420C
:106F90004F525400496E76616C6964206F70636F64
:106FA00064652072656365697665643A203078258A
:106FB000782E0000526571756573742068616E6487
:106FC0006C696E6720636F6D706C6574652E2052FE
:106FD0006573756C743A20307825780038B10549AE
:106FE00001600549416001210172002070470E20B7
:106FF00070470000FD6F0F0035700F0010B50C00DA
:1070000001464FF0110007D02278052A05D2DFE8AB
:1070100002F00F050D0F0F000E2010BD084600F006
:107020006FF80028F9D10221217010BD112010BD88
:10703000082010BD0246082041B10B78022B04D174
:10704000022A05D0032A00D1112070470E20704774
:10705000002003220A70704770B50F480024D0F852
:107060005C11491C03D1D0F89C01401C11D00B4885
:107070000421008801EB004009A101F0AFFA4FF4B0
:107080007F25284601F050FC57220349284601F08D
:1070900063FC204670BD0000EC7F002044590020B6
:1070A00045726173696E672073657474696E677386
:1070B0002070616765206164646974696F6E616CDA
:1070C00020646174612E000010B528B11C220349B0
:1070D000FAF7DAF9002010BD0E2010BD9CF10F0068
:1070E00010B5064C00221821201DFDF763F9216818
:1070F000814201D1012010BD002010BD9CF10F0084
:1071000070B50C4D0400D5F89C0105F5CE7503D083
:10711000401C03D0082070BD0E2070BD0022182135
:10712000201DFDF747F9206007222146284629DF68
:1071300070BD000000F00F00002258210148FDF74B
:1071400039B90000F07F00202DE9F0411F4C0546C1
:10715000042620881EA106EB004001F03FFA2846D5
:10716000FFF756FC02004FF0010504D0208821A152
:1071700005EB004023E04FF4DC78424628492948DB
:10718000FAF782F9274F3868401C04D0FFF7D4FF84
:107190003968814218D0208823A106EB004001F015
:1071A0001DFA41461F48FAF797F900207D6000F06C
:1071B00061F8020008D0208823A105EB004001F00F
:1071C00011FA0320BDE8F0810020FBE740590020C0
:1071D00043616C6C696E67206E72665F6466755F92
:1071E00073657474696E67735F696E697428292E9C
:1071F0002E2E00006E72665F6466755F666C61734A
:10720000685F696E69742829206661696C6564200D
:1072100077697468206572726F723A202578000071
:1072200000F00F00EC7F0020526573657474696E86
:107230006720626F6F746C6F616465722073657430
:1072400074696E67732E00006E72665F6466755FA8
:10725000666C6173685F777269746528292066615E
:10726000696C65642077697468206572726F723A20
:10727000202578002DE9F04105464FF4DC773A46A9
:1072800021492248FAF73AF9214C0426002820889F
:1072900006EB004015D01FA101F0A0F920881A4A82
:1072A00006EB004020A101F09DF9002201211648C3
:1072B000FFF746FB012668B1208823A106EB0040BA
:1072C0001DE02AA101F08AF90DB10020A847002095
:1072D000BDE8F081FFF730FF0C493A460860A1F5A0
:1072E000DC70FAF7D1F82B463A4630490648FFF7EA
:1072F000D7FB0028ECD020882DA106EB004001F040
:107300006DF90320E4E7000000F00F00EC7F00209F
:107310004059002057726974696E672073657474F0
:10732000696E67732E2E2E0045726173696E672039
:107330006F6C642073657474696E67732061743A4E
:107340002030782530387800436F756C64206E6F7C
:107350007420657261736520746865207365747448
:10736000696E677320706167652100004E65772044
:1073700073657474696E67732061726520696465F2
:107380006E746963616C20746F206F6C642C20775D
:1073900072697465206E6F74206E65656465642E15
:1073A00020536B697070696E672E0000347E002078
:1073B000436F756C64206E6F7420777269746520FA
:1073C000746865204446552073657474696E6773EC
:1073D00020706167652100004FF480507047000005
:1073E0002DE9F04782461548154FDFF85880C01B3D
:1073F000C608B8F800104FF0040909EB0140002559
:10740000324611A101F0EEF8002411E007EBC400B0
:10741000416850468847050009D0B8F800102B464F
:1074200009EB0140224612A101F0E3F802E0641CDE
:10743000B442EBD32846BDE8F087000038CD0F00FA
:1074400030CD0F006C5900205368757474696E67F5
:1074500020646F776E207472616E73706F727473D4
:107460002028666F756E643A2025642900000000AC
:107470004661696C656420746F2073687574646F0D
:10748000776E207472616E73706F72742025642C35
:10749000206572726F722025640000002DE9F047AC
:1074A00082461448144FDFF85480C01BC608B8F851
:1074B00000104FF0040909EB01400025324610A1ED
:1074C00001F090F8002410E057F834105046884737
:1074D000050009D0B8F800102B4609EB0140224600
:1074E00010A101F086F802E0641CB442ECD32846F7
:1074F000BDE8F08738CD0F0030CD0F006C5900206B
:10750000496E697469616C697A696E672074726129
:107510006E73706F7274732028666F756E643A2094
:10752000256429004661696C656420746F20696E6A
:10753000697469616C697A65207472616E73706FC9
:1075400072742025642C206572726F72202564008D
:1075500070B5114D114CA86B30B103F0CBFD18B1D3
:10756000686A08B1012000E000202070FEF708FEE4
:1075700018B10B498E20FBF73DFF4023094A0A4909
:107580000A48FEF747FD002805D0BDE870400449D1
:107590009620FBF72FBF70BDEC7F002038580020ED
:1075A000B8C10F0010B70F005084002090B70F0033
:1075B0002DE9F041134C07460D46E06BA26B012606
:1075C0004119914209D910480121008801EB00407E
:1075D0000EA101F003F8032610E00A492A465C31A7
:1075E00008443946F9F750FFE06B064A2844E06347
:1075F000403229463846FCF7DDFE20643046BDE8BF
:10760000F0810000EC7F002048590020496E697429
:1076100020636F6D6D616E64206C617267657220AE
:107620007468616E2065787065637465642E00000F
:1076300070B505004FF0010404D0B5F5807F03D983
:1076400004240CE003240AE006490020064E0870DA
:107650002021306306F13800F9F73EFFB56320467C
:1076600070BD000038580020EC7F00202DE9F04765
:10767000304C0E468046D4E90E010125DFF8B89063
:107680002F46814208D0B9F800002CA107EB00403A
:1076900000F0A4FF082549E0DFF8BCA09AF800003C
:1076A00030B1FEF7AFFEC8F80000606A30603DE020
:1076B00003F020FD88B3294890F89C1009B901789F
:1076C00059B3041D0021C8F80010316090F89C30B7
:1076D0000A462BB1214C90F83811A03404F19902DC
:1076E00094F8590003F048FB054601281ED1201DDF
:1076F00000F0B8F80546012818D18AF80070314624
:10770000201D03F005FF054601280FD14246201D2C
:10771000316803F0BBFE054608E0FFE7B9F800005A
:107720000FA107EB004000F059FF05252846BDE8F2
:10773000F0870000EC7F0020485900204578656301
:107740007574652077697468206661756C7479203A
:107750006F6666736574000038580020A4810020AD
:107760004661696C656420746F206465636F64654D
:1077700020696E6974207061636B6574000000009D
:107780000148007870470000385800202DE9F04784
:1077900080462748264D894690F89C00012608B16E
:1077A000A43500E008350A4641462846FDF792FA1E
:1077B000204C002760B195F8550058B100F0010148
:1077C000C0F340024346284602F0FCFEC8B114E074
:1077D000172617E00120E06217480421008801EB1A
:1077E000004016A100F0FAFE276295F88F0010B154
:1077F00095F8900008B96868A060A06CC4E9099089
:1078000004E005260B482430FEF70CFE0948202131
:107810003830F9F761FE0748FF22F4215C30F9F7B0
:1078200054FEC4F8488030462763BDE8F087000066
:10783000A4810020EC7F002048590020496E766129
:107840006C69646174696E67206F6C64206170702C
:107850006C69636174696F6E20696E2062616E6B22
:1078600020302E002DE9F04104004FF0010503D136
:1078700040497F20FBF7BEFD94F854003E4E01279F
:1078800040B194F8550050B1012808D0022806D024
:10789000032804D0308839A107EB004064E01CB90C
:1078A00034496720FBF7A6FD94F86D00032807D044
:1078B000308838A107EB004000F090FE142556E018
:1078C00094F88F00B84618B194F8900000284ED173
:1078D000207A58B1E068022734280CD0308832A1D1
:1078E00007EB004000F07AFE112540E0318808EBFC
:1078F000014032A138E0204603F0AEF918B12078FB
:1079000050B394B907E0308830A107EB004000F095
:1079100065FE12252BE017498C20FBF76BFD2078C4
:1079200018B914498D20FBF765FD94F855002B49D3
:1079300068B101280BD06068C968884217D83088C0
:1079400027A107EB004000F049FE10250FE060681A
:10795000896888420BD2F2E794F85500012806D0D6
:10796000318808EB014023A100F038FE0F2528469E
:10797000BDE8F08100C20F004C590020496E7661CD
:107980006C6964206669726D7761726520747970C4
:10799000652E0000496E76616C69642068617368C9
:1079A00020747970652E00004661756C74792048EA
:1079B000572076657273696F6E2E00004E6F2048F7
:1079C000572076657273696F6E2E000053442072E3
:1079D0006571206E6F74206D65742E00EC7F002041
:1079E00046572076657273696F6E20746F6F206CD6
:1079F0006F772E0046572076657273696F6E206D23
:107A0000697373696E672E000FB438B5040003D133
:107A100010A11C20FBF7EEFC606918B90DA11D2018
:107A2000FBF7E8FC206818B90AA11E20FBF7E2FC6E
:107A3000606818B907A11F20FBF7DCFC0599002935
:107A400005D006A800906A46204600F045F838BCEC
:107A50005DF814FB2E2E5C2E2E5C2E2E5C2E2E5CE2
:107A60002E2E5C65787465726E616C5C66707269EE
:107A70006E74665C6E72665F667072696E74662E96
:107A80006300000010B5040003D107A10B20FBF731
:107A9000B1FCA268002A05D0D4E904032168984704
:107AA0000020A06010BD00002E2E5C2E2E5C2E2E1D
:107AB0005C2E2E5C2E2E5C65787465726E616C5C3B
:107AC000667072696E74665C6E72665F667072690B
:107AD0006E74662E630000002DE9FC4791460C464B
:107AE0005FEA000804D183A14FF49F70FBF782FC8A
:107AF000D8F8140020B97FA14FF4A070FBF77AFCEE
:107B0000D8F8000020B97BA140F24110FBF772FCCD
:107B1000D8F8040020B977A14FF4A170FBF76AFCF4
:107B2000002C76D014F8011B39B125290ED040461F
:107B3000FCF734FB20780028F4D198F80C000028DA
:107B400067D04046BDE8FC47FFF79CBF00200122FC
:107B500021782B291BD02D2902D0302908D102E011
:107B600040F0010001E040F00200641C002AEFD167
:107B700000252A290ED02178A1F130020A2A11D23B
:107B800005EB850201EB4205641C303DF1E740F056
:107B90000400EAE7D9F800100B1DC9F800300968A5
:107BA000641C0D44217800232E290BD114F8011FE9
:107BB000A1F130020A2A05D203EB830201EB420352
:107BC000303BF3E76C290DD068290BD0692921D00F
:107BD0000BDC252918D0582931D063290ED064290F
:107BE00015D117E014F8011FECE7702969D073294B
:107BF00032D075291BD0782909D120E0D9F80000AE
:107C0000011DC9F8001001784046FCF7C7FA641C52
:107C100090E76CE0D9F800100A1DC9F80020096847
:107C2000CDE900500A224046FDF7AEFAEFE7D9F859
:107C300000100A1DC9F8002009680A2206E0D9F8D8
:107C400000100A1DC9F8002009681022CDE9005073
:107C5000404603F0C1FBDAE7D9F8001000270A1DFF
:107C6000C9F800200E68C00705D112E04046761C16
:107C70007F1CFCF793FA31780029F7D104E020212A
:107C800040466D1EFCF78AFABD42C0D9002DF6D1E0
:107C9000BDE74EB13046F9F72AFC074604E0202143
:107CA00040466D1EFCF77AFABD4206D9002DF6D18A
:107CB00003E04046761CFCF771FA31780029F8D1D0
:107CC000A5E7D9F80000011DC9F8001005683021AA
:107CD0004046FCF763FA78214046FCF75FFA08203B
:107CE0000021CDE90001034610222946B0E7BDE896
:107CF000FC8700002E2E5C2E2E5C2E2E5C2E2E5C21
:107D00002E2E5C65787465726E616C5C667072694B
:107D10006E74665C6E72665F667072696E74665FC2
:107D2000666F726D61742E63000000002DE9F041F2
:107D30001E4615460F46040003D11DA17820FBF70F
:107D400059FB206818B91AA17920FBF753FB1DB91C
:107D500017A17A20FBF74EFB39462046FBF776F851
:107D600040B939462046FBF771F818B910A17D20BB
:107D7000FBF740FB60683946026820466A43FBF720
:107D80006EF858B960683946026820466A43FBF7C6
:107D900066F818B906A17F20FBF72CFB2068334654
:107DA0002A46D0F810C039462046BDE8F041604769
:107DB0002E2E5C2E2E5C2E2E5C2E2E5C2E2E5C63C8
:107DC0006F6D706F6E656E74735C6C6962726172F8
:107DD0006965735C6673746F726167655C6E726609
:107DE0005F6673746F726167652E630070B51646C7
:107DF0000C46050003D108A12F20FBF7FBFA1CB9A4
:107E000005A13020FBF7F6FA2C603146284622689F
:107E1000BDE87040104700002E2E5C2E2E5C2E2EEA
:107E20005C2E2E5C2E2E5C636F6D706F6E656E74B3
:107E3000735C6C69627261726965735C6673746F9E
:107E4000726167655C6E72665F6673746F7261679C
:107E5000652E63002DE9F04128B1016819B1C969A7
:107E6000BDE8F04108470D4D0D480024461B14277E
:107E70000DE000BF04EB840005EB8000016829B130
:107E8000C969884710B10120BDE8F081641CB6FBC8
:107E9000F7F0A042EED80020F6E7000010590020CD
:107EA00024590020044801214174007A08B10020BF
:107EB000704701207047000058870020012801D03A
:107EC000032808D10449002201284A7400D0002068
:107ED000087402F03DBC70475887002070B5014619
:107EE000022801D0032943D1224C207A00283FD018
:107EF000012831D002282FD11F4800230229006811
:107F000002D0032928D119E0E360027912B1012AD5
:107F100022D10BE0D0E90565721B142A00D314228C
:107F20002A4482614569AA420ED015E00169491CC4
:107F30000161426991420FD1237213E0E268521C41
:107F4000E260082A08D9E360237202290AD00D21D1
:107F5000FCF74FFE02F0F2FB607C28B1BDE87040F8
:107F600000F01EBF0021F3E7BDE8704002F0F0BB57
:107F700070BD000058870020A05800202DE9F8436C
:107F80001D46089F16468846040003D12AA1622098
:107F9000FBF730FA1EB928A16320FBF72BFA206803
:107FA00018B925A16420FBF725FA1DB922A1652087
:107FB000FBF720FA60684068B5FBF0F100FB115157
:107FC00041B1B5FBF0F100FB115018B11AA16820C6
:107FD000FBF710FA4046FAF733FF38B94046FAF794
:107FE0002FFF18B914A16B20FBF704FA3046FAF7FB
:107FF00027FF38B93046FAF723FF18B90EA16C20D5
:10800000FBF7F8F92A4641462046FAF728FF48B917
:108010002A4641462046FAF722FF18B906A16D20EC
:10802000FBF7E8F9009720682B463246C7684146BF
:108030002046B847BDE8F8832E2E5C2E2E5C2E2EEF
:108040005C2E2E5C2E2E5C636F6D706F6E656E7491
:10805000735C6C69627261726965735C6673746F7C
:10806000726167655C6E72665F6673746F7261677A
:10807000652E63002DE9FF411C46DDE90A781546AF
:108080000E46684600F010F846EA450141EA8401D0
:1080900041EA072242EA0841009A00EB8200C0F858
:1080A0000017BDE8FF81000010B5044600683028C5
:1080B00004D308A140F2A110FBF79CF92068202806
:1080C00002D24FF0A04010BD00F01F0020600C480D
:1080D00010BD00002E2E5C2E2E5C2E2E5C2E2E5CF3
:1080E0002E2E5C6D6F64756C65735C6E7266785C69
:1080F00068616C5C6E72665F6770696F2E68000005
:108100000003005010B504460068302804D308A1CD
:1081100040F2A110FBF76EF92068202802D24FF040
:10812000A04010BD00F01F0020600C4810BD0000F2
:108130002E2E5C2E2E5C2E2E5C2E2E5C2E2E5C6D3A
:108140006F64756C65735C6E7266785C68616C5C9C
:108150006E72665F6770696F2E68000000030050E2
:1081600038B501240090684631B1FFF79DFF0099B2
:108170008C40C0F8084538BDFFF796FF00998C4049
:10818000C0F80C4538BD000030B5104B014600204A
:108190001C69224609E0157A854205D1401C0A284F
:1081A000F7DB4FF0FF3030BD5268002AF3D1421C9C
:1081B000F9D008721A6922B152684A601A6951608E
:1081C00030BD002219614A6030BD00006C9800206B
:1081D0007047FAF755BC704708B5034A0092402330
:1081E000024A00F005F808BD29AD0F006C87002099
:1081F000F0B595B01C4615460F4608461A9E00F08D
:1082000071FB182109A8F9F767F90E96CDE9095411
:108210000023082203A9384600F079FB0598069050
:10822000BDF81000ADF81C00BDF81200ADF81E003E
:1082300000208DF821000398082600F00300012893
:1082400002D0022818D032E003983346850AC0F3E2
:10825000C2008DF8200003980FA9C0F38314A20078
:10826000384600F054FB09A8009006AB22460FA93F
:10827000284600F093FA1AE00398840DC0F3C20078
:108280008DF82000082C01D2254600E00825334651
:108290002A460FA9384600F03AFB2E44641B09AB6E
:1082A00006AA29460FA800F0CDF9002CEAD13846DD
:1082B00000F01EFB15B0F0BD0A4A012902EBC00018
:1082C00007D0022907D0032907D0042907D00020AE
:1082D000704702207047042070470079704740794A
:1082E0007047000038CD0F0010B5FFF772FF042172
:1082F0000648FFF749FF002803DA05491B20FBF772
:1083000079F802490120487210BD0000AC580020E5
:108310005CC70F002DE9F04F8DB0FBF74FFF18B190
:1083200000200DB0BDE8F08F794E0020B061BFF3A2
:108330004F8FA6F580544FF0000960680190A56842
:10834000284004EB800008E021680198814201D8B0
:108350006160E5E7284004EB80000C3001A9FCF7E0
:1083600067FF0028F0D105AAA046019901EA05049B
:1083700008EB8403491CDB6842F82030401C019163
:108380000228F2D3059800F00300022802D0012849
:108390004CD0A6E005985022810D8A46B2EB905F42
:1083A00000D850210C4664F39F500590083159487D
:1083B00000F04FFA070075D000F094FA4B460822FF
:1083C00005A9384600F0A9FA019909F1080B2940DE
:1083D000681A8000001D844221D94F4D30B1C2B2CD
:1083E00008EB8101201A91460C3104E02946E2B2E3
:1083F000002591462846C4B25B46384600F08DFA07
:108400000BEB090325B122462946384600F085FAD0
:1084100001990AF1030001EB900001903BE008EBA9
:1084200081015B46224638460C31EFE70598C0F3E0
:108430008310062800D30620059960F38911C1F343
:108440008310801C05918100324800F002FA070079
:1084500047D000F047FA4B46082205A9384600F0FD
:108460005CFA09F1080900240FE001984B4600EA84
:108470000501401C08EB81010190042238460C31B3
:1084800000F04BFA09F10409641C0598C0F383104D
:10849000A042EAD837B13469B06968B1384600F013
:1084A00027FA2FE01DE0607A012804D122682046D7
:1084B0003946126890476468002CF4D1384600F0C1
:1084C00017FA00208DF800006846FAF703FFB0693C
:1084D00010B90199C8F804109DF80000FAF746FF9A
:1084E00010E0346904E021682046896888476468A0
:1084F000002CF8D109480221008801EB004008A1B6
:1085000000F06CF8FBF75AFE80F0010009E700006C
:108510006C98002000CE0F00788800206C59002055
:108520004261636B656E647320666C757368656425
:10853000000000002DE9F84F8146264FD01C15465B
:108540008A46800800226946BE68FBF7D1FDB8B3B1
:10855000009CB846A01C0090B9683040091A8F00F2
:108560003F1DBD4208EB800002D82A46514608E074
:108570003A4651460C30F8F787FF1648EA1B0AEBDB
:1085800007010C30F8F780FF4FEA1947FCF724F990
:1085900047EA0042601C304008EB8000344008EBA2
:1085A0008401C260C8684FF6C07269F3C500904389
:1085B00065F39F5020F00300801C20F00400C86089
:1085C000054890F8200001E0FFF7A4FE0028FBD149
:1085D000BDE8F88F6C8800206C98002000231A46B4
:1085E00002F030BD08B5012300926A4602F02AFD70
:1085F00008BD1CB5CDE9002302236A4602F022FD26
:108600001CBD3EB5069C8DE81C0003236A4602F0A3
:1086100019FD3EBD7FB5DDE908458DE83C0004232A
:108620006A4602F00FFD7FBD70B586B00DF1280CD3
:108630009CE870008DE87C0005236A4602F002FD8C
:1086400006B070BD2DE9F0470E4680461C469246A6
:1086500008293ED894F80C90002020731946104643
:1086600002F012F80025B54206D218F805201AA12A
:108670002046FFF7C9F903E019A12046FFF7C4F926
:108680006D1C082DEFD317A12046FFF7BDF900257B
:10869000B54210D218F80570F8F7F2FE0068C05D18
:1086A00010F03E0F01D03A4600E02E220EA12046E7
:1086B000FFF7AAF903E00DA12046FFF7A5F96D1C0D
:1086C000082DE5D301222146504601F05DFF84F8D4
:1086D0000C90BDE8F08700002025303278000000C3
:1086E000202020007C000000256300002000000006
:1086F000104910B540F2FF308860002008604860E3
:1087000001F580518861486181F820000A4800F035
:10871000EDF800280CD1094809490A4B401AC10854
:10872000002002E023F82000401C8842FAD30020F9
:1087300010BD00006C88002000CE0F00E8CD0F00B7
:1087400038CD0F002459002002480349401AC008C0
:1087500070470000E8CD0F0038CD0F0013B5684614
:10876000FCF704FF08B100201CBD0248009950F836
:1087700031001CBD38CD0F0070B5074801250469D4
:1087800080F8205005E065722168204649688847D6
:108790006468002CF7D170BD6C9800202DE9FF476C
:1087A00081460C9D00200C462F7B28739846164668
:1087B0002946184601F068FF072E42D2DFE806F08E
:1087C00004090F161F2A360049462846FFF71CF9F0
:1087D00037E0494628462268FFF716F931E0D4E928
:1087E000002349462846FFF70FF92AE0A0680090C9
:1087F000D4E9002349462846FFF706F921E0D4E9E9
:108800000201CDE90001D4E9002349462846FFF7DB
:10881000FBF816E004F1080007C88DE80700D4E96A
:10882000002349462846FFF7EFF80AE004F1080064
:108830000FC88DE80F00D4E9002349462846FFF70A
:10884000E3F800222946404601F09EFE2F73BDE862
:10885000FF872DE9F041858A80462D1F4819C01CED
:10886000B0FBF5F0C6B24046FCF712FF041E19D06B
:108870000020207101206071E58000272546761ECA
:10888000C4F800800BE04046FCF702FF60B161795C
:10889000491C6171286005467F1CC0F80080B74202
:1088A000F1D32046BDE8F081204600F002F8002018
:1088B000F8E72DE9F041457901466B1E002201E001
:1088C0000968521C9A42FBD30F680146002605E056
:1088D00038460C68FCF742FF2146761CAE42F7D3BF
:1088E000BDE8F0810121001DFCF7ABBEFCF77EBFA7
:1088F00010B504460121001DFCF7C4FE10F0FF0F67
:1089000004D12046BDE81040FFF7D3BF10BD38B5F5
:1089100001240094FCF7E0FD38BD38B50024009434
:10892000FCF7DAFD38BD0000094902220A60BFF3F6
:108930006F8FBFF34F8F0A1D106006480268002A30
:10894000FCD000200860BFF36F8FBFF34F8F7047DC
:1089500004E5014000E4014070B50E4C01232360A2
:10896000BFF36F8FBFF34F8F00230B4D08E000BFA5
:1089700051F8236040F823602E68002EFCD05B1C69
:108980009342F5D300202060BFF36F8FBFF34F8F6A
:1089900070BD000004E5014000E4014020B103493E
:1089A00009680160002070470E20704780BC0F00EE
:1089B0002DE9FE4306460D460846FFF7EFFF002867
:1089C0007ED18046CDF80080CDF8048001240620B9
:1089D0008DF80060ADF80400CDF808808DF80240F5
:1089E000694620202A6869DF3F4F40B100F0A2FBB2
:1089F000024638883D4904EB0040FFF7F3FDCDF80F
:108A000000808DF801408DF80280CDF80480CDF80B
:108A100008808DF80380694640202A6869DF40B1EC
:108A200000F088FB02463888314904EB0040FFF72C
:108A3000D9FDCDF800808DF80060F720ADF8020078
:108A4000CDF80480CDF80880694623202A6869DFC4
:108A500040B100F06FFB02463888264904EB004025
:108A6000FFF7C0FDCDF80080CDF80480CDF8088078
:108A70008DF800404646694601202A6869DF40B10A
:108A800000F058FB024638881B4904EB0040FFF712
:108A9000A9FD4FF4B0600090019602966946A120AE
:108AA0002A6869DF40B100F045FB02463888134967
:108AB00004EB0040FFF796FD00960196029600E059
:108AC00010E08DF800606946A0202A6869DF40B197
:108AD00000F030FB02463888094904EB0040FFF7FC
:108AE00081FD0020BDE8FE8374590020ACC90F0051
:108AF000F4C90F0040CA0F000CC90F0058C90F007D
:108B0000B8C80F002DE9F0410446D0F8008060DFBE
:108B10002168194D074641451CD92888022606EBD5
:108B2000004016A1FFF75AFD2888424606EB004098
:108B30001EA12368FFF75DFDF006D0F80C01216847
:108B4000800200F10050421A288825A106EB00405F
:108B5000FFF748FD012467B1384600F0EBFA024602
:108B600028882AA104EB0040FFF73CFD3846BDE809
:108B7000F0812E480470F9E774590020496E73752E
:108B80006666696369656E742052414D20616C6C44
:108B90006F636174656420666F722074686520532A
:108BA0006F66744465766963652E00004368616E84
:108BB0006765207468652052414D2073746172743A
:108BC000206C6F636174696F6E2066726F6D203008
:108BD00078257820746F20307825782E00000000EA
:108BE0004D6178696D756D2052414D2073697A65CC
:108BF00020666F72206170706C69636174696F6E5A
:108C000020697320307825782E00000073645F623D
:108C10006C655F656E61626C65282920726574758C
:108C2000726E65642025732E000000000B59002031
:108C300030B51848ADF5017D0078002826D04FF4F6
:108C4000FA7400BFADF8004280A9684661DF38B110
:108C500005281BD00DF5017DBDE83040FAF718BAA4
:108C60006D460D497DA800F0F1F809E07DA800F0FF
:108C7000D5F8D0E90021284690477DA800F024F9D6
:108C80007DA800F0CBF80028DCD0EFE70DF5017DE2
:108C900030BD00000B59002084BC0F00F8B5134C08
:108CA0002078C0B10120A07002F008F8112814D07B
:108CB000022002F01FF800258DF800506846FAF7F0
:108CC00009FB11DF064625709DF80000FAF74EFB00
:108CD0002EB13046F8BD0820F8BD0020F8BDA570C3
:108CE00002F05CF9032002F005F8F6E708590020CD
:108CF0007CB5194C207808B108207CBD0120A070FB
:108D0000002001F0DBFF112819D0002001F0F2FF54
:108D100012480026006801908DF800606846FAF756
:108D2000D9FA0F4901A810DF05000AD000202070F1
:108D30009DF80000FAF71AFB2DB128467CBD0020F3
:108D40007CBD0120F3E7A670667002F043F90120B4
:108D500001F0D0FFF3E700000859002018BC0F0015
:108D600035300F000EB50A49684600F06FF808E08C
:108D7000684600F047F8D0E900108847684600F0E0
:108D8000A3F8684600F03EF80028F1D10EBD0000BF
:108D900034BC0F00014800787047000008590020DB
:108DA0000548817819B1007818B1FFF777BF08201E
:108DB0007047FFF79DBF0000085900201FB56846A7
:108DC0004BDF30B1052819D004B0BDE81040FAF7E8
:108DD0005FB90B4901A800F039F809E001A800F0DB
:108DE00029F8D0E900210098904701A800F06CF81C
:108DF00001A800F01FF80028E1D0EFE71FBD000038
:108E0000A0BC0F0010B5040003D103499E20FAF75F
:108E1000F1FAA06810BD000064C80F0010B504008E
:108E200003D103499E20FAF7E5FAA06810BD0000BF
:108E300064C80F0010B5040003D103499E20FAF75F
:108E4000D9FAA06810BD000064C80F0070B50D46C7
:108E5000040003D108492A20FAF7CCFA1DB90649C3
:108E60002B20FAF7C7FA2560286860602046BDE825
:108E7000704000F003B800001CC30F0010B50400E0
:108E800003D110490D20FAF7B5FA206818B90D4939
:108E90000E20FAF7AFFA606818B90A490F20FAF7FE
:108EA000A9FAD4E900104A68904201D1002004E0F8
:108EB000D0E900239A4202D01046A06010BD0830CD
:108EC0006060F0E71CC30F0010B5040003D1124925
:108ED0003D20FAF78FFA206818B90F493E20FAF7BB
:108EE00089FAA068002815D0216889680844A06024
:108EF000606818B908494D20FAF77CFAD4E90101F5
:108F00004268914206D1083060602046BDE81040BA
:108F1000FFF7B4BF10BD00001CC30F0070B50D46B5
:108F2000060003D10BA11420FAF764FA1DB909A1B8
:108F30001520FAF75FFA746804E0B2682946904792
:108F400018B1246820680028F7D1206828602560BF
:108F500070BD00002E2E5C2E2E5C2E2E5C2E2E5C04
:108F60002E2E5C636F6D706F6E656E74735C6C69D2
:108F7000627261726965735C736F72746C69737429
:108F80005C6E72665F736F72746C6973742E6300CB
:108F900010B5040003D103A13D20FAF72BFA206895
:108FA00010BD00002E2E5C2E2E5C2E2E5C2E2E5C14
:108FB0002E2E5C636F6D706F6E656E74735C6C6982
:108FC000627261726965735C736F72746C697374D9
:108FD0005C6E72665F736F72746C6973742E63007B
:108FE00010B5040003D103A13720FAF703FA606833
:108FF000006810BD2E2E5C2E2E5C2E2E5C2E2E5C5C
:109000002E2E5C636F6D706F6E656E74735C6C6931
:10901000627261726965735C736F72746C69737488
:109020005C6E72665F736F72746C6973742E63002A
:1090300010B5040003D105A12B20FAF7DBF9616814
:109040000868002801D002680A6010BD2E2E5C2E30
:109050002E5C2E2E5C2E2E5C2E2E5C636F6D706F40
:109060006E656E74735C6C69627261726965735C63
:10907000736F72746C6973745C6E72665F736F7217
:10908000746C6973742E630070B50C46050003D1CF
:109090000BA14320FAF7AEF91CB909A14420FAF755
:1090A000A9F90021686806E0A24203D121680160A5
:1090B000012103E010460268002AF5D1084670BD80
:1090C0002E2E5C2E2E5C2E2E5C2E2E5C2E2E5C63A5
:1090D0006F6D706F6E656E74735C6C6962726172D5
:1090E0006965735C736F72746C6973745C6E7266BD
:1090F0005F736F72746C6973742E63000C4A10B5E1
:1091000002F594730EE0991AC91001EBD171491060
:1091100002EBC1010C68844201D90B4602E005D282
:1091200001F108029A42EED3002010BD486810BD3C
:10913000C8BA0F0000B5FFF7E1FF002800D10148D1
:1091400000BD0000B4BA0F002DE9F04104461348F9
:10915000134BC01A0C21B0FBF1F6A0694FF0FF31A0
:1091600010F8022C02B92169002011E000EB400543
:1091700003EB85052F68974209D14F1C02D06F6819
:109180008F4204D194E80F00AD68A84703E0401C6B
:10919000B042EBD301202060BDE8F08154CE0F0037
:1091A00048CE0F0002480068002800D00120704718
:1091B0000004014070B50C46050003D10D49D920CB
:1091C000FAF718F91CB90B49DA20FAF713F90A482B
:1091D0000421008801EB004008A1FFF7FFF91249C4
:1091E0000320C96888476869FEF722FAFBF756FD35
:1091F000607070BDE0BF0F003C59002048616E6494
:109200006C65204E52465F4446555F4F505F4F425B
:109210004A4543545F4352454154452028636F6D8E
:109220006D616E64290000002858002070B50C465E
:1092300020B9154940F20110FAF7DCF824B91249B7
:109240004FF48170FAF7D6F8104D042610A1288843
:1092500006EB0040FFF7C2F91849081FFEF706FAAF
:10926000FBF71CFD6070012805D10020FEF702F815
:1092700010B10A20607070BD288811A106EB004073
:10928000BDE87040FFF7AAB9E0BF0F003C590020CD
:1092900048616E646C65204E52465F4446555F4F90
:1092A000505F4F424A4543545F45584543555445E6
:1092B0002028636F6D6D616E6429000030580020B6
:1092C00057726974696E672076616C696420696E93
:1092D000697420636F6D6D616E6420746F20666CBD
:1092E0006173682E0000000070B50D46040003D1C4
:1092F0001749E720FAF77EF8206918B91449E820E1
:10930000FAF778F8A08A18B91149E920FAF772F843
:109310001DB90F49EA20FAF76DF80E4804210088BC
:1093200001EB00400CA1FFF759F9A18A2069FEF773
:109330003FF9FBF7B3FC68702846FBF721F8E168BA
:10934000002903D02069BDE87040084770BD0000C7
:10935000E0BF0F003C59002048616E646C65204EF0
:1093600052465F4446555F4F505F4F424A45435413
:109370005F57524954452028636F6D6D616E6429B3
:109380000000000030B587B00C4605461822184989
:109390006846F8F779F8207B0195164D8DF80000A6
:1093A000012806D0022812D006281CD1607B049028
:1093B00019E01148FEF714F8A888E880607B049053
:1093C000617CD4F80E0061F31F6005900BE00B4840
:1093D0000421008801EB004009A1FFF7FFF8B4F871
:1093E0000D00A880E8806846FDF7B4FC07B030BDEA
:1093F00038B90F000858002030CD0F003059002038
:109400005365742072656365697074206E6F74694A
:10941000660000002DE9F0410B4E0D460427308810
:109420000AA107EB0040FFF7D9F8114C308811A1D1
:1094300007EB0040A36C226DFFF7DBF8A06CA8607F
:10944000206D6860BDE8F0813C59002048616E6481
:109450006C65204E52465F4446555F4F505F435205
:10946000435F47455420286461746129000000006F
:10947000EC7F00204F66667365743A25642C2043A8
:1094800052433A3078253038780000002DE9F84F03
:109490003E4C81460D462088042707EB00403CA146
:1094A000FFF79CF8FEF76CF901264FF0080AC8B1E7
:1094B000D9F814204FF00308DAB13F493F481305AB
:1094C0001CD0436DD1F808C01344634516D02088E2
:1094D0003BA106EB004000BFFFF780F885F8018054
:1094E000BDE8F88F20883FA106EB0040FFF776F833
:1094F0001EE0208849A106EB0040EDE7B2F5805F51
:1095000007D920884CA106EB0040FFF767F86F7081
:10951000E6E7436DD1F808C003EB0208E0450AD93D
:10952000CDF800C020884D4906EB0040FFF769F8F0
:1095300085F801A0D4E74264C26C036503638046EA
:109540008264D9F81400002200F6FF704FEA103C44
:10955000486861461844FDF7F3F940B1208840A1FE
:1095600006EB0040FFF73AF805206870B8E7D8F836
:1095700048100091208840A107EB0040D8F85030F7
:10958000D8F84420FFF73DF8AAE700003C59002036
:1095900048616E646C65204E52465F4446555F4F8D
:1095A000505F4F424A4543545F4352454154452022
:1095B000286461746129000028580020EC7F002095
:1095C0004F626A6563742073697A65206D75737480
:1095D000206265207061676520616C69676E6564F3
:1095E0000000000043616E6E6F74206372656174E9
:1095F000652064617461206F626A656374207769B5
:1096000074686F75742076616C696420696E697422
:1096100020636F6D6D616E64000000004F626A65CB
:1096200063742073697A652063616E6E6F74206263
:109630006520302E00000000496E76616C69642060
:1096400073697A6520666F72206F626A6563742041
:1096500028746F6F206C6172676529006CBF0F0002
:109660004572617365206F7065726174696F6E20F9
:109670006661696C656400004372656174696E6758
:10968000206F626A65637420776974682073697AF1
:10969000653A2025642E204F66667365743A203043
:1096A00078253038782C204352433A2030782530C2
:1096B000387800002DE9F041154D07460E46288800
:1096C000042101EB004013A1FEF788FF1B4CD4E9F5
:1096D0001401626C431A9A420BD02888012101EBD5
:1096E000004017A1FEF785FF082070700120BDE83B
:1096F000F08100216164A16CE1646065002138465D
:1097000000F032F817490420C96888470020EEE7C6
:109710003C59002048616E646C65204E52465F449F
:1097200046555F4F505F4F424A4543545F45584549
:10973000435554452028646174612900EC7F002062
:10974000496E76616C696420646174612E2065786D
:109750007065637465643A2025642C20676F743AE1
:1097600020256400285800202DE9F041044686B0E9
:109770000020FEF76FFB224E012758B1214A182125
:109780002046F9F7A1FC020036D030881EA107EB75
:1097900000402FE0182227496846F7F775FE264853
:1097A000264D4FF00408006DA968884211D1318818
:1097B00008EB014022A1FEF711FFD5E90101FDF7F9
:1097C000E5FF8DF80100FBF769FA8DF80100254DE2
:1097D00002E08DF801700025D4E901126846904737
:1097E00015B12846FDF746FD31889DF8012008EBAC
:1097F00001401DA1FEF7F6FE06B0BDE8F0810000B5
:109800003C59002069970F004661696C65642074BB
:109810006F207363686564756C65206F626A656349
:109820007420657865637574653A20307825782EE4
:1098300000000000F8B90F00EC7F0020285800203D
:10984000506F737476616C69646174696F6E206FB8
:1098500066206669726D7761726520696D61676502
:109860002E000000119A0F00526571756573742007
:1098700068616E646C696E6720636F6D706C65748F
:10988000652E20526573756C743A20307825780007
:10989000F8B50C4D0C46042628880BA106EB0040B9
:1098A000FEF79CFE124813A1826CA260036DB00209
:1098B0006360E0600090288806EB0040FEF7A1FEA0
:1098C000F8BD00003C59002048616E646C65204E74
:1098D00052465F4446555F4F505F4F424A4543549E
:1098E0005F53454C4543542028646174612900004E
:1098F000EC7F0020637263203D20307825782C2097
:109900006F6666736574203D20307825782C206D55
:1099100061785F73697A65203D2030782578000092
:109920002DE9F041264F05460E463888042101EB0B
:10993000004024A1FEF752FEFDF722FF98B12B4C08
:10994000D4E91401401AA98A0844616C88420CD9F0
:109950003888012101EB004025A1FEF73FFE0320DE
:109960007070BDE8F0810820FAE72749206B49684C
:109970004718E86820B925494FF4E070F9F73AFD37
:10998000D5E90331AA8A3846FDF78AF820B1D5E92E
:109990000310BDE8F0410847A98A206B134A084428
:1099A0002063A98A206D483208442065A98A286965
:1099B000FAF700FDA064B060206D7060D1E7000090
:1099C0003C59002048616E646C65204E52465F44ED
:1099D00046555F4F505F4F424A4543545F57524987
:1099E000544520286461746129000000EC7F002048
:1099F0005772697465207265717565737420746F30
:109A00006F206C6F6E67000028580020E0BF0F00C9
:109A1000074810B50088042101EB004005A1FEF7BE
:109A2000DDFD11490620C968BDE810400847000067
:109A30003C590020416C6C20666C617368206F702B
:109A400065726174696F6E73206861766520636FFB
:109A50006D706C657465642E2044465520636F6D8F
:109A6000706C657465642E0028580020FEF784FE33
:109A7000FEF750FC0028FBD10D4E64254FF47A47C9
:109A8000741C3846A0476D1EFAD10A480068C0070A
:109A900000D000BEBFF34F8F0648E4380168064A85
:109AA00001F4E06111430160BFF34F8F00BFFDE798
:109AB00050B70F00F0ED00E00400FA0510B50446C1
:109AC000074804212246008801EB004005A1FEF76B
:109AD00089FD2146BDE810400748FBF73FBE000066
:109AE0003059002046726565696E6720627566664A
:109AF0006572202570000000E8CD0F002DE9F047C9
:109B00002F4F05464FF0040938880C464E4609EBA6
:109B100000402CA1FEF762FD38882A7C06EB00404D
:109B200031A1FEF75FFD4FF44051374B4A680120E9
:109B30004FF002089A4200D10220344E326A012AC4
:109B400000D1401C4FF0010C84F801C02A7C1AB1EE
:109B50000025012A09D01BE084F80480F068A06089
:109B60002B48E060C0F57E200FE0D1F804809845D6
:109B70000ED125710878142801D9486900E0002029
:109B8000A0604FF48050E06088682061BDE8F087F5
:109B9000824208D284F804C0B068A060FCF71CFCC4
:109BA000E060B069F1E7398809EB014019A1FEF7DF
:109BB00015FDFF202071A560E5602561E6E7000046
:109BC0003C59002048616E646C65204E52465F44EB
:109BD00046555F4F505F4649524D574152455F567B
:109BE000455253494F4E00004669726D7761726568
:109BF00020696D6167652072657175657374656450
:109C00003A20256400000000DBE5B151EC7F002024
:109C100000100F004E6F2073756368206669726DC7
:109C20007761726520696D616765000030B58A1DD6
:109C30008B79083187B0022B33D153888489A342B2
:109C40002FD1127A012A2CD1184C0DF1040C3CCCE6
:109C50008CE83C000A89ADF80C204A890C3104914B
:109C60001249ADF80E208039114C096A0591CDF8E2
:109C700018D0018A05AA6088ADDF18B96846FAF7DE
:109C800005F938B10020ADF8080001A96088B0DFFF
:109C900050B106E040F2FD10ADF8080001A960885F
:109CA000B0DF002007B030BD0120FBE750B90F0046
:109CB0000858002070B506468C1DC888B18888B049
:109CC000884229D11948FBF7E3FC0500184825D044
:109CD000F42100910088042101EB004063892A46A9
:109CE00014A1FEF78EFC628904F10C012846F7F7F7
:109CF000CBFB1822174901A8F7F7C6FB029605957A
:109D00006089ADF8180001A8FDF724F8002803D0F9
:109D100029460648FBF722FD08B070BD00880221E5
:109D200001EB00400CA1FEF759FCF5E7E8CD0F0070
:109D30003059002042756666657220257020616387
:109D40007175697265642C206C656E20256420280D
:109D50002564290060B90F0063616E6E6F74206125
:109D60006C6C6F63617465206D656D6F72792062D4
:109D70007566666572210000F8B50D461446064604
:109D8000694600F052FA00280ED0009AFF2A0AD83D
:109D9000501C824207D869780223B3EB911F02D08E
:109DA0002979814201D20020F8BD2270611C304621
:109DB00000F080FBF8BD114600F0D6B8114600F067
:109DC000E3B8F8B50C4615460646694600F02DFA8C
:109DD00000280CD0009A501C904207D361780223CF
:109DE000B3EB911F02D02179814201D20020F8BD4E
:109DF0002946304600F05EFB009A0021A954F8BDC8
:109E00002DE9FF410C468E6817460546694600F06D
:109E100023FB00280ED0A06800280BD060783A46BB
:109E2000C0F3011002283146684606D000F0DAF887
:109E30000199696004B0BDE8F08100F086F8F7E7A9
:109E40007CB50D461446694600F08FF9002820D0F5
:109E50002879082806D0042809D002280AD0012829
:109E60000CD015E0DDE90001C4E900010AE000982A
:109E7000206006E0009800B2208002E0009840B226
:109E80002070C117DDE9002350405940084301D03C
:109E900000207CBD01207CBD7CB50D461446694682
:109EA00000F09EF9002820D02879082807D000214A
:109EB000042809D002280AD001280CD014E0DDE9DA
:109EC0000001C4E9000109E00098206006E0009864
:109ED00080B2208002E00098C0B22070DDE900234B
:109EE00050405940084301D000207CBD01207CBD7A
:109EF0007CB50D461446694600F072F9002821D061
:109F00002979082908D00098C21704290BD0022902
:109F10000DD001290ED014E0DDE90002C4E90002F1
:109F20000146134609E0C3170146206005E001B26F
:109F3000218001E041B22170CB17414053401943C9
:109F400001D000207CBD01207CBD70B50D460646C9
:109F500014461146284600F09AFA22462946304611
:109F6000BDE8704000F03EB838B50C4604226946A2
:109F700000F0A0FA002806D09DF80310009861F3C5
:109F80001F602060012038BD1CB50C4608226946C0
:109F900000F090FA002824D09DF801109DF80020D0
:109FA0009DF80230080E42EA012242EA034240EAEA
:109FB00013409DF803309DF8041040EA1320084335
:109FC0009DF8051042EA036240EA01209DF8061060
:109FD00040EA01409DF8071040EA0160C4E9002012
:109FE00001201CBD2DE9F04F04469DB000200090DB
:109FF000064601904FF0FF3A0AA800F069F94FF0C9
:10A00000010BE94682E012AB05AA06A9204600F042
:10A01000C9F850B10AA8059900F06BF960B10B9826
:10A02000407810F0300F53D060E09DF848000028D1
:10A0300070D11DB0BDE8F08F0598B04242D30B9DA2
:10A040000AAE0B98407800F00F00082812D0304676
:10A0500000F066F90B98A842F3D156460599B14233
:10A0600030D3D4F8088009919DF8181008910E9902
:10A070000D6820E00B980678F0E729680F682FB18B
:10A08000DDE9083229462046B84711E01194896875
:10A09000DDE90872097891420CD1294617A8FBF72F
:10A0A0006BF985F80CB017AA39461198FAF7DFF961
:10A0B0000028BED0AD6815B1A1684145DDD0A168CA
:10A0C000414523D19DF81810204600F02FFA1BE0DF
:10A0D0000C9840280AD200F01F010BFA01F00C99ED
:10A0E0004A0959F82230034349F82230E5682DB176
:10A0F0000AAB9DF8182020460599A8470AAA9DF8A2
:10A1000018102046FAF7B3F9002892D0A06800286A
:10A110007FF479AFDDE90B0445780AA800F000F977
:10A120000028F7D115F0300F03D10B98007800B15B
:10A13000641CC4B10020494605E000BF51F820204E
:10A14000521C0ED1401CB0EB541FF7D3600959F8D4
:10A15000201004F01F00C0F120022AFA02F0814210
:10A1600001D0002065E7012063E71CB50C46694675
:10A1700000F036F8002814D0DDE90002C10709D04C
:10A1800051084FEA30006FEA00026FEA0100C4E9AB
:10A19000002004E051084FEA3000C4E900014FF00C
:10A1A00001001CBDF8B507460020187008700E4667
:10A1B00010601C4615466946384600F036F8012105
:10A1C00040B1009850B1C10800F00700296030701C
:10A1D0000120F8BDB86808B10020F8BD2170FBE788
:10A1E0002DE9F8430026884681463446354604E08A
:10A1F000402E02D30020BDE8F8836946484600F0AF
:10A2000085F90028F7D09DF80070324607F07F00EE
:10A21000C10FF7F726F929430443F61D0D4638060A
:10A22000E6D4C8E900410120E5E7F8B50E46074647
:10A23000694600F06BF900280AD09DF8004020061E
:10A2400016D5072504F07F0403E0202D01D300205C
:10A25000F8BD6946384600F059F90028F8D09DF855
:10A26000001001F07F00A8400443ED1D0806ECD467
:10A2700001203460F8BD000059680A4A896891429B
:10A280000ED1D0E901120848491C521EC0E9011242
:10A2900006480421008801EB004005A1FEF7A2B9A1
:10A2A00070470000DCB70F003858002048590020E4
:10A2B00050423A20496E6974207061636B65742066
:10A2C00064617461206C656E3A20256400000000B2
:10A2D000C26000230160C0E901138B781A44026157
:10A2E00091F903301A4442610878002800D0012017
:10A2F000704770B545680E46044660680178B14203
:10A3000006D1407800F00F00082801D0012070BD70
:10A31000204600F005F86068A842EED1002070BD2C
:10A3200030B541680A785AB101F10C0343600A7BE9
:10A3300042B14C780A79C4F30115032D07D00BE024
:10A34000002030BDC2680168FFF7C2FFF8E75D7802
:10A35000C5F30115032D07D00225B5EB141F09D154
:10A360004C7914FB02F209E08D7804690022641B29
:10A37000046103E0B5EB941F00D10422497811F089
:10A38000300F02D18168491C81609C7801692144A9
:10A390001144016193F9032011444161012030BD52
:10A3A00030B54168002487B0497801F00F02082ACF
:10A3B00011D08A091ED00222B2EB911F09D1026985
:10A3C000C1F301110229146001D0032901D14069B0
:10A3D000047007B030BD0069056808E02C73294699
:10A3E0006846FAF7C9FF6846FFF7DAFFAD68002D47
:10A3F000F4D1EEE7C1F30111012912D00229E6D010
:10A400000329E4D04268517801F00F0107290BD0ED
:10A41000916881B11279006907B0BDE83040F7F763
:10A4200033B841690C70EDE70169906807B0BDE889
:10A43000304000F02CB81179006907B0BDE8304019
:10A44000F7F74AB810B5034B002408C080E816009F
:10A4500010BD000081410F0038B50D460446694625
:10A46000FFF7E3FE00280BD0D4E90002D4E9021381
:10A47000C5E90002C5E902130098814201D200201B
:10A4800038BDA860A168081AA060012038BD00B5D9
:10A490000A4687B001466846FFF71AFF002807D032
:10A4A0006846FFF77DFF6846FFF73AFF0028F7D1BF
:10A4B00007B000BD7FB514460546A9B9124A286801
:10A4C000904208D110E0102269462846FFF7F2FFBB
:10A4D000002807D0103C102CF5D8224669462846A3
:10A4E000FFF7E8FF04B070BDA868A04201D20020C9
:10A4F000F8E72B682246284698470028F2D0A8683B
:10A50000001BA8600120EDE781410F0010B5044653
:10A510008068002809D02368012220469847002837
:10A5200003D0A068401EA060012010BD38B50024F3
:10A5300039B1012912D0022912D005291DD00020DD
:10A5400038BD0546012269462846FFF7B3FF90B1A2
:10A550009DF800000006F5D4012038BD08220DE06A
:10A5600005466946FFF761FE28B100212846009A9A
:10A57000FFF7A0FF38BD204638BD0422BDE83840B3
:10A580000021FFF797BF000010B50C46017A05299E
:10A5900008D0407A38B1084808A102682046FDF783
:10A5A00033FA00E01AB106A12046FDF72DFA204645
:10A5B000BDE81040FDF766BAE4580020257300009E
:10A5C0000D0A00002DE9F047284D9946164604462D
:10A5D00081B3284F09F50052DFF894C038885368DA
:10A5E000A16D4FF0010808EB0040634501D02249FE
:10A5F0000AE093684A1EC2F30B02891A41F6FF7201
:10A6000011448B4205D21D49FDF7E8FF0020BDE84B
:10A61000F0874846FAF74AFE90B13888022101EBEC
:10A6200000401749FDF7DAFF2EB110481830FBF74C
:10A63000F9FE06E00CE0398808EB01401149E3E738
:10A640000EB1AC2000E0A520E862A06D686301E0D7
:10A65000AA20E8623EB194F88F0010B194F89000FF
:10A6600008B96068E8600120D1E70000EC7F0020B5
:10A67000DBE5B1514859002020C10F00B4C00F00E4
:10A6800074C10F0070C00F0038B5C3880D46044672
:10A6900033B114A0009015A216A12846FDF7B4F915
:10A6A000217A05291CD0607A48B1A088FDF704FE04
:10A6B000164951F8202016A12846FDF7A5F9A088D3
:10A6C0000021FEF74BF803461049207A143951F85F
:10A6D000202001B02846BDE830400EA1FDF794B916
:10A6E00038BD00001B5B306D000000001B5B313B80
:10A6F00033316D0025734C6F67732064726F707017
:10A700006564202825642925730D0A00E45800207B
:10A71000257300003C25733E2025733A200000007D
:10A72000EFF30580C005C00D01D001207047EFF3A5
:10A73000148040F30000401C7047000003480249A9
:10A740000068FAF751BF0000A458002084BA0F0037
:10A750002DE9F041224C0025224E207A012730B904
:10A760002148311D0068FAF74AFF306038B10220F5
:10A7700020723168087928B101281CD114E0656085
:10A78000BDE8F081D1E90503C01A142800D31420D4
:10A79000B7EB900F01D2820800E001220869C96876
:10A7A0001844194429DF03E0D1E90301084428DFF4
:10A7B00058B1112812D003213068FAF71AFA25721D
:10A7C0006560BDE8F041FFF7B9BF207C0028D7D114
:10A7D000BDE8F04100210220FDF780BB2772CFE7E2
:10A7E00058870020A058002084BA0F0010B5074CED
:10A7F000201DFAF723FF002806D1607C002803D132
:10A80000BDE81040FFF7A4BF10BD0000588700202E
:10A8100010B510461A46F6F737FE002010BD10B5E9
:10A8200010461A46F6F730FE002010BD2DE9F04123
:10A830001E681C461546074621B1012918D0052976
:10A8400023D119E000202060401C2060B0421CD8B9
:10A85000012229463846FFF72DFE002806D015F8BC
:10A86000010B000601D52068EEE70120BDE8F0816C
:10A8700008200246186002E00420024618602946BB
:10A880003846BDE8F041FFF715BE0020EEE770B591
:10A8900016460A460446C11C104600F07BFD0546DC
:10A8A00061193046C91C00F075FD284470BD0000D8
:10A8B00003B5094A85B0D2E91612CDE9001207495D
:10A8C0008989ADF8001006A9CDE90210044869464F
:10A8D0004088AEDF07B000BDD0B80F00D86D0020B3
:10A8E0000858002008467047084670472DE9F04197
:10A8F0008046FAF75AF81A4D0026F0B1686828B178
:10A9000068684068696820F07F40486000F08EFB0E
:10A91000040012D04FF080776068B84203D220461E
:10A9200000F03AFC03E0606820F07F406060204661
:10A93000FEF72EFB08B10446EEE700214046F9F78A
:10A9400055FF28B1686818B1686800F025FC6E6092
:10A95000404600F085FC4046BDE8F04100F002B8FA
:10A96000545800202DE9F041214C0746002600BF35
:10A9700000F05CFB90B341686068406862685AB15F
:10A980006268002A28D0884226D96068007E18B103
:10A9900061681848FEF7C2FA00F04EFB42680546AF
:10A9A00013484FF47A7300210830FAF71FF830B1DA
:10A9B0000D2807D010499C20F8F71CFDD8E76068E7
:10A9C00020B106E0284600F0E7FBD1E73846F9F76A
:10A9D000F1FF6560002ECBD1BDE8F081FFE7606834
:10A9E0000028F9D13846BDE8F041F9F7F1BF000081
:10A9F0005458002030BA0F004CC20F002DE9F05F10
:10AA0000FCF7EAFCDFF8CC80334D0427D8F830207F
:10AA1000D8F8346000EB020BB01A411EC1F30B01F1
:10AA2000401A00F6FF7A28882CA107EB0040D8F8DE
:10AA30004840FDF7D3FD42F20400324900594FF07F
:10AA40000109884208D0298809EB01402EA1FDF7B1
:10AA5000C5FD0320BDE8F09FD8F830000444B042A3
:10AA600007D1288835A107EB0040FDF7B7FD00208E
:10AA7000F0E7D0B904F500500178142901D94069F4
:10AA800000E000203249B0FBF1F34FF4405002786F
:10AA9000142A01D9406900E00020B0FBF1F22888B7
:10AAA0002CA107EB0040FDF7A4FD082352462146E8
:10AAB0005846FAF75DFA040007D0298809EB0140EF
:10AAC0002FA1FDF78BFD2046C4E7BDE8F05F002015
:10AAD000FCF7D0BBEC7F00206C590020456E7465FC
:10AAE00072206E72665F626F6F746C6F6164657204
:10AAF0005F6466755F73645F636F6E74696E7565BE
:10AB000000000000DBE5B151536F75726365206191
:10AB100064647265737320646F6573206E6F742054
:10AB2000636F6E7461696E20612076616C69642068
:10AB3000536F66744465766963652E0053442061E3
:10AB40006C726561647920636F70696564000000F0
:10AB500040420F005570646174696E672053442E43
:10AB6000204F6C64205344207665723A2025642C73
:10AB7000204E6577207665723A202564000000003B
:10AB80004661696C656420746F20636F707920661C
:10AB900069726D776172652E0000000070B50F4C10
:10ABA0000421208801EB00400DA1FDF717FDFFF700
:10ABB00025FF05004FF0010604D0208810A106EB08
:10ABC000004007E0F8F722FC050006D0208812A11B
:10ABD00006EB0040FDF702FD284670BD6C590020D1
:10ABE000456E746572206E72665F6466755F73642D
:10ABF0005F626C5F636F6E74696E75650000000064
:10AC000053442B424C3A20534420636F70792066A2
:10AC100061696C656400000053442B424C3A204249
:10AC20004C20636F7079206661696C656400000078
:10AC300070B50346002002464FF4405409E000BFBF
:10AC400053F82250A689B54201D1012070BD521C93
:10AC5000D2B28A42F4D370BD10B5040003D11549B5
:10AC60003220F8F7C7FB4FF4405013494068884240
:10AC700015D1217C04F1140009B162694AB994F834
:10AC8000552012B1012A08D10DE0012905D96269C8
:10AC90001AB9BDE81040FFF7CBBF012010BD207CE2
:10ACA00018B1606908B1002010BD20780028F4D1E7
:10ACB00010BD000000C20F00DBE5B1513EB50446F7
:10ACC0000B496846FEF7C2F80AE06846FEF79AF8B4
:10ACD000D0E900212046904740B16846FEF7F4F8DD
:10ACE0006846FEF78FF80028EFD13EBD11203EBD2B
:10ACF0001CBC0F003EB504460A496846FEF7A6F89C
:10AD000009E06846FEF77EF8D0E90021204690472A
:10AD10006846FEF7D9F86846FEF774F80028F0D1C7
:10AD20003EBD000028BC0F002DE9F041140088460C
:10AD300018D000250E4F032608EB050122460020FF
:10AD4000F7F7A0FE0544241A40B93878002809D046
:10AD500008494FF47A408847761E05D001203870A4
:10AD6000002CE9D1BDE8F08100203870FAE700003E
:10AD7000A858002001BC0F00FEB5474C20200290CF
:10AD800020880F460325164605EB004043A1FDF73A
:10AD900025FC46B1208805EB00406FB149A1FDF7C5
:10ADA0001DFC1620FEBD2088022101EB00404BA1B6
:10ADB000FDF714FC1320FEBD4D4F4EA1BA68FDF700
:10ADC00011FC02A95848CDE90001D7E901235749F0
:10ADD000A0F58A70FBF770F910B93278402A01D0DB
:10ADE0000A20FEBD5048711C4038F6F74DFB208804
:10ADF0004FA105EB0040FDF7F1FB4B4840214038E7
:10AE0000CDE90001A0F14801474AA0F5BC70029BC2
:10AE1000FBF71AF90200208836D0012101EB00402F
:10AE200048A1FDF7DFFB2088042505EB00404EA17B
:10AE3000FDF7D4FB20883C4905EB00404022403917
:10AE4000FDF778FB20884BA105EB0040FDF7C6FB22
:10AE50000298354982B2208805EB0040FDF76AFB75
:10AE6000208846A105EB0040FDF7B8FB2088402272
:10AE700005EB00404449FDF75DFB00BFFDF74AFAD2
:10AE80000028FBD10520FEBD05EB00403FA1FDF7EA
:10AE9000A5FB0120FEBD0000485900205369676EE4
:10AEA00061747572652072657175697265642E20B2
:10AEB000436865636B696E67207369676E6174755B
:10AEC00072652E00496E76616C6964207369676EE5
:10AED0006174757265207479706500004E6F20731F
:10AEE00069676E617475726520666F756E642E0099
:10AEF0003858002043616C63756C6174696E67201B
:10AF0000696E6974207061636B6574206861736831
:10AF10002028696E6974207061636B6574206C65AC
:10AF20006E3A202564290000D88400209CB70F00C9
:10AF3000566572696679207369676E6174757265AA
:10AF4000000000005369676E617475726520666168
:10AF5000696C656420286572725F636F64653A206E
:10AF600030782578290000005369676E6174757226
:10AF7000653A0000486173683A0000005075626CE1
:10AF80006963204B65793A0010B70F00496D61671E
:10AF900065207665726966696564000010B51620E3
:10AFA000F7F73CFF48B10A4882684FF4800152B17C
:10AFB000016821F48001016010BDBDE8104042F23B
:10AFC0000100F8F765B84FF0E020C0F8801110BD1F
:10AFD0007085002010B51620F7F720FFA0B11148AA
:10AFE00090F800044009082811D280B101280ED041
:10AFF00004280CD00C4882684FF480016AB10168C3
:10B0000041F48001016010BD42F2010001E042F212
:10B010000200BDE81040F8F73BB84FF0E020C0F860
:10B02000001110BD16E000E0708500200148FDF71A
:10B03000D7BF000030BA0F000148FDF7F9BF00008C
:10B0400030BA0F002DE9F84FDFF89C80934689460F
:10B0500006461F46012269461846D8F80850F9F7F7
:10B0600047F8B0B3009800210446C246801C08E0AF
:10B0700000EA05025BF821300AEB8202401C491C01
:10B08000D360B942F4D3C846B946370CF9F7A4FBEC
:10B090008346FDF759FBB84204D8144940F28310A7
:10B0A000F8F7A8F9601C28400AEB80002C4047EA1A
:10B0B0000B420AEB8401C260C86866F3C50069F3FD
:10B0C000891068F39F2020F00300401C20F004004A
:10B0D000C860074890F8200002E000BFFDF71AF9A9
:10B0E0000028FBD1BDE8F88F6C880020B0C70F00A6
:10B0F0006C9800201FB5134800F15C01826B684614
:10B10000FFF7A0F910489DE80E0080E80E000E49F8
:10B110000E48104AC8600E490020486088600E49F9
:10B120000948FEF712FF10B1012004B010BD0B4812
:10B130000121008801EB004009A1FDF74FFA002032
:10B14000F3E70000EC7F00204084002079A20F008C
:10B1500038580020A4810020A8B80F0048590020CA
:10B1600048616E646C65723A20496E76616C696400
:10B170002070726F746F636F6C20627566666572A3
:10B18000206D5F70625F73747265616D0000000016
:10B19000002800D00047704770B50446C06818B951
:10B1A0000F496120F8F726F90E4800250078A0B174
:10B1B0009CB1207E88B1D4E903108847A06850B1C3
:10B1C000217E41B161680844606021460648FDF770
:10B1D000A5FE012501E000202076284670BD000074
:10B1E0004CC20F005458002030BA0F0070B5164CF6
:10B1F0002078002827D1154801680125C1F30041B6
:10B2000031B913490D600168C1F300410029FAD03A
:10B21000F8F704F808B1F7F73BFF0E4A00210E4893
:10B22000F7F7DEFF18B10D492E20F8F7E3F80A48CA
:10B23000084A0121001DF7F7D3FF18B10749332051
:10B24000F8F7D8F8257070BDF857002018040040B2
:10B250000800004091B10F0088B70F0058BD0F00E3
:10B260002DE9F843244D814669462868FAF7C7F965
:10B27000044600274FF00108204E39E0207820B125
:10B2800001281BD002282AD122E06068017E31BB50
:10B2900080F818804846F9F7B0FA014660684268BD
:10B2A000511A174A914203D9416821F07F41416008
:10B2B000114861680830FDF731FE10E06168706880
:10B2C000814200D177600C480830FDF7DDFE06E0D2
:10B2D000FFF7B2FE08B10776FAE786F80080694604
:10B2E0002868FAF781F969462868FAF788F9044668
:10B2F000002CC3D1BDE8F88328BA0F0054580020B1
:10B3000017FCFF00F8B50B4C0D4606466946206851
:10B31000FAF75FF958B10670456069462068FAF798
:10B3200079F910B10448F9F72FFB0020F8BD04208B
:10B33000F8BD000028BA0F005C58002070B5154613
:10B340000C460646FFF752FF3046F7F7B1FF18B13B
:10B350000F494320F8F74EF8002C17D0610CE0039A
:10B360004FF4FA72801841F1000152000023F6F701
:10B3700047F801462A463046F7F776FF002805D001
:10B38000BDE8704002494A20F8F734B870BD0000AB
:10B3900058BD0F000870020A4A70020C8A70000E35
:10B3A000C87004207047000010B50248FAF73DF954
:10B3B000002010BD8858002010B514210448F6F76D
:10B3C0008BF804480068FAF7E9F8002010BD000087
:10B3D0005887002084BA0F002DE9F05F8346DDE92D
:10B3E0000A4A994690460D460846012703E000BFE9
:10B3F000B0FBF8F07F1C4045FAD2B94500D94F4662
:10B400005FEACA7012D18CB15FEA8A7002D5B9F1D5
:10B41000000F01D0202607E0302605E031465846CF
:10B42000641EF8F7BBFE0CB1A742F7D35FF001062C
:10B43000B9F1010F02D9A9F1010903E0B5FBF6F05A
:10B44000404502D306FB08F6F2E7DFF83C9000BF68
:10B45000B5FBF6F000FB165519F800105846F8F742
:10B460009DFEB6FBF8F6002EF2D15FEACA7009D055
:10B47000002C07D0A74205D220215846641EF8F7B9
:10B480008DFEF5E7BDE8F09F46BA0F002DE9F041CB
:10B49000084601241646254600212B460A46FAF79F
:10B4A000CBFF0C4F38B138880BA105EB0040FDF7FE
:10B4B00095F804240BE0FAF7A5FF306039880422E0
:10B4C00002EB014302460BA11846FDF78BF820461C
:10B4D000BDE8F0814859002043616E2774206669F9
:10B4E0006E6420726F6F6D20666F7220757064617C
:10B4F00074650000577269746520616464726573D5
:10B50000732073657420746F20307825303878008C
:10B510002DE9F0410F24002790F85520184E012501
:10B520001AB990F86430012B06D0D30707D090F8F1
:10B530005630012B02D002E0876E0DE0876D920736
:10B540000AD590F85C20012A06D1026E0D48C0F59C
:10B550007E239A4204D817444FB101240F600CE0B7
:10B56000308809A105EB0040FDF743F8042430883A
:10B570000DA105EB0040FDF731F82046BDE8F08154
:10B580004859002000100F00424C2073697A652052
:10B5900028256429206F766572206C696D69742096
:10B5A0002825642900000000496E697420706163D9
:10B5B0006B657420646F6573206E6F7420636F6EAB
:10B5C0007461696E2076616C6964206669726D775A
:10B5D0006172652073697A650000000030B100680F
:10B5E0000549884205D048F20250704748F20150A0
:10B5F00070470020704700006E52464870B5FDF756
:10B60000D1FD002811D00020084A094B094C012126
:10B61000166801FA00F52E4203D004EB8005C5F848
:10B620000036401CC0B20728F2D370BD08050140A7
:10B630003546526E00000140084810B54078002899
:10B640000BD007480321008801EB004005A1FCF75F
:10B65000C5FFBDE81040FFF7D1BF10BDFA5700206D
:10B660002C590020496E7465726E616C20666565A8
:10B670006400000000207047002070472DE9FC4165
:10B6800080461C4617460E460C48089DF9F7D6FF23
:10B6900010B11120BDE8FC81A20839463046FDF703
:10B6A0005BF90648F9F7C1FF33463A4601214046A7
:10B6B000CDE90045F9F782FA0020EBE78858002031
:10B6C0002DE9F84F114D884681461E4617466946BA
:10B6D000DDF828A02868F9F77CFF040013D01C21AE
:10B6E000F5F7FAFE00202071C4F80090C4E9048642
:10B6F000C4E902A769462868F9F78CFFFFF776F8D6
:10B700000020BDE8F88F0420FBE7000084BA0F009A
:10B7100065FC2BF816DA019ADE75D4A847719621DC
:10B720001C875569105ABE04578FD2B0299456B859
:10B73000CA0363D635C64DA7819FEFA7D2ECB7F3F6
:10B7400007FF80AF7A3B4C19B891C5143CE8766D81
:10B750000338FDD870470D0E0F100B0C18190000A0
:10B760000338FDD870470000000000000000000012
:10B77000000000000000000000000000FFFFFFFFCD
:10B780000000000000000001C0570020DC5700202E
:10B79000480000000020400000000000C9420F00E7
:10B7A000D9420F0075420F00200000000000000089
:10B7B0000000000000000000010100000100000086
:10B7C0000000000002050000210000000000000051
:10B7D000000000000000000000000000011104FC57
:10B7E0000400000000000000021104FC040000003E
:10B7F00000000000032104FC041000000000000011
:10B80000041101FF0100000000000000051102FE0C
:10B810000400000000000000061104FC0400000009
:10B8200000000000071104FC0400000000000000FC
:10B83000081701FF22000000B8B70F00091001FF30
:10B8400001000000B4B70F0000000000000000007D
:10B8500000000000011101FF0100000000000000D5
:10B86000021702FE94000000DCB70F000000000089
:10B870000000000000000000010700009800000028
:10B8800054B80F0002010000010000000000000099
:10B89000030500004100000000000000000000005F
:10B8A0000000000000000000011704FC98000000E8
:10B8B00054B80F00021704FCDC00000078B80F0039
:10B8C0000000000000000000000000000000000078
:10B8D000001103000011130002000000010000002D
:10B8E0000338FDD870470C000C000000580200001F
:10B8F0000200000000000000020000000000000044
:10B900009C6D002009000000000000000000000005
:10B9100001000000000000002800000000000000FE
:10B920000000000000010000000001000000000015
:10B930000000000000000000000000000000000007
:10B9400029360F0000000000000000000000000089
:10B9500002000000000001000000000000000000E4
:10B96000080000000000000029360F00BD9A0F00FB
:10B9700000000000000000000400000000000000C3
:10B9800000000000000000000000000000000000B7
:10B9900000000000000000000000000000000000A7
:10B9A000F40000000000000018000000000000008B
:10B9B0000000000000000000000000000000000087
:10B9C0000000000000000000000000000000000077
:10B9D000170000000000000050EADA308883B89FAA
:10B9E000604F15F30000C98E020000000000000047
:10B9F0000000000000000000040000000000000043
:10BA00000000000000000000000000000000000036
:10BA10000001000000000000000000000000000025
:10BA20000000000000000000645800200000070033
:10BA30000000000078580020A5430F00000000001F
:10BA40000338FDD870473031323334353637383922
:10BA5000414243444546000000100000040000003D
:10BA60000100000045510F00A9B30F0011A80F00FD
:10BA70007DB60F00294B0F00E5A80F0075B60F002B
:10BA80008D520F008C5800200010000004000000B0
:10BA90000100000051510F00B9B30F001FA80F00A3
:10BAA000C1B60F00714B0F00E9A80F0079B60F0067
:10BAB0009D520F00556E6B6E6F776E206572726FC0
:10BAC0007220636F6465000000000000E8C60F008C
:10BAD0000100000094C50F000200000088C30F00A1
:10BAE0000300000008C60F00040000005CC60F0041
:10BAF000050000003CC50F0006000000D8C40F0080
:10BB00000700000044C60F000800000050C50F00E9
:10BB100009000000B4C50F000A000000D0C60F00E5
:10BB20000B00000070C30F000C00000068C50F0080
:10BB30000D00000038C70F000E00000034C60F00D3
:10BB40000F00000070C60F0010000000A4C60F0018
:10BB5000110000004CC70F001200000020C70F00AA
:10BB600013000000BCC60F0080000000F0C40F00EE
:10BB7000810000002CC40F0082000000ECC30F0005
:10BB800083000000CCC30F008400000008C40F0035
:10BB90008500000014C50F00860000001CC60F00C1
:10BBA00090000000B8C40F0091000000ACC30F006B
:10BBB000920000007CC50F000082000084C60F00C8
:10BBC00001820000D0C50F0002820000ECC50F000A
:10BBD0000084000048C40F0001840000F4C60F0078
:10BBE0000284000090C40F00038400006CC40F00A6
:10BBF000D9810F00D7810F00D1810F000000000014
:10BC00000338FDD87047000020CE0F0028CE0F006B
:10BC100000000000000000000100000708BC0F0049
:10BC200018BC0F000800000040BC0F0050BC0F0003
:10BC30000800000050BC0F0060BC0F0008000000AE
:10BC400040CE0F0048CE0F000000000000000000B2
:10BC500030CE0F0040CE0F000000000000000000BA
:10BC600000000000000000000000000000000000D4
:10BC700018CE0F0020CE0F000000000000000000D2
:10BC8000B857002060BC0F0080BC0F000800000007
:10BC900028CE0F0030CE0F00000000000000000092
:10BCA00090BC0F00A0BC0F0008000000F19E0F0028
:10BCB000999E0F00419E0F00B79D0F00BD9D0F0084
:10BCC000799D0F00C39D0F00019E0F000000000032
:10BCD000004040404040404040404141414141409F
:10BCE0004040404040404040404040404040404054
:10BCF00040050202020202020202020202020202E3
:10BD000002202020202020202020200202020202E7
:10BD1000020290909090909010101010101010103F
:10BD2000101010101010101010101010020202024B
:10BD3000020288888888888808080808080808088F
:10BD4000080808080808080808080808020202028B
:10BD500040000000D1BC0F002E2E5C2E2E5C2E2E3B
:10BD60005C2E2E5C2E2E5C636F6D706F6E656E7434
:10BD7000735C6C69627261726965735C626F6F7427
:10BD80006C6F616465725C6E72665F626F6F746C1B
:10BD90006F616465725F6466755F74696D65727307
:10BDA0002E6300002E2E5C2E2E5C2E2E5C2E2E5C22
:10BDB0002E2E5C636F6D706F6E656E74735C6C6954
:10BDC000627261726965735C626F6F746C6F6164DB
:10BDD00065725C6E72665F626F6F746C6F616465D2
:10BDE000725F66775F61637469766174696F6E2EE6
:10BDF0006300000043524320636F6D70757461747B
:10BE0000696F6E206661696C656420666F7220637D
:10BE10006F70696564206170703A2073726320638B
:10BE200072633A203078253038782C207265732080
:10BE30006372633A20307825303878004120536FA0
:10BE4000667444657669636520686173206A7573FA
:10BE500074206265656E20616374697661746564DF
:10BE60002E2049742773206C696B656C7920746887
:10BE7000617420616E206170706C69636174696FB8
:10BE80006E2077696C6C20636F6D6520696D6D65E0
:10BE900064696174656C790052656365697665648F
:10BEA00020424C455F47415454535F4556545F45CB
:10BEB000584348414E47455F4D54555F5245515593
:10BEC0004553542028726571756573743A20256452
:10BED0002C207265706C793A202564292E000000B0
:10BEE0002E2E5C2E2E5C2E2E5C2E2E5C2E2E5C6357
:10BEF0006F6D706F6E656E74735C6C696272617287
:10BF00006965735C626F6F746C6F616465725C62AB
:10BF10006C655F6466755C6E72665F6466755F62B1
:10BF20006C652E63000000006E72665F6673746F4E
:10BF3000726167655F777269746528616464723DD8
:10BF400025702C207372633D25702C206C656E3D2E
:10BF50002564206279746573292C20717565756577
:10BF60002075736167653A2025640000437265613E
:10BF700074696E6720746865206F626A65637420F7
:10BF8000776974682073697A65203078253038784D
:10BF900020776F756C64206F766572666C6F7720A2
:10BFA0006669726D776172652073697A652E204FBC
:10BFB0006666736574206973203078253038782080
:10BFC000616E64206669726D776172652073697A4B
:10BFD00065206973203078253038782E0000000005
:10BFE0002E2E5C2E2E5C2E2E5C2E2E5C2E2E5C6356
:10BFF0006F6D706F6E656E74735C6C696272617286
:10C000006965735C626F6F746C6F616465725C64A8
:10C0100066755C6E72665F6466755F7265715F6897
:10C02000616E646C65722E63000000002E2E5C2E23
:10C030002E5C2E2E5C2E2E5C2E2E5C636F6D706F30
:10C040006E656E74735C6C69627261726965735C53
:10C05000626F6F746C6F616465725C6466755C6E50
:10C0600072665F6466755F7574696C732E63000039
:10C070004D616A6F7220534420757064617465204D
:10C08000627574206E6F20424C2E2041626F727474
:10C0900020746F2061766F696420696E63617061DE
:10C0A0006369746174696E672074686520424C2E00
:10C0B0000000000054686520536F6674446576691B
:10C0C00063652073697A6520696E207468652069EC
:10C0D0006E666F2073747275637420697320746F59
:10C0E0006F20736D616C6C20636F6D70617265643D
:10C0F0002077697468207468652073697A65207296
:10C1000065706F7274656420696E2074686520695B
:10C110006E697420636F6D6D616E642E00000000A7
:10C1200054686520536F667444657669636520645E
:10C130006F6573206E6F7420636F6E7461696E201B
:10C14000746865206D61676963206E756D626572E4
:10C15000206964656E74696679696E672069742008
:10C160006173206120536F66744465766963652E40
:10C1700000000000496E76616C69646174696E67E5
:10C180002061707020626563617573652069742039
:10C19000697320696E636F6D70617469626C65208C
:10C1A000776974682074686520536F667444657697
:10C1B0006963652E000000002E2E5C2E2E5C2E2E54
:10C1C0005C2E2E5C2E2E5C636F6D706F6E656E74D0
:10C1D000735C6C69627261726965735C626F6F74C3
:10C1E0006C6F616465725C6466755C6E72665F64D8
:10C1F00066755F76616C69646174696F6E2E630049
:10C200002E2E5C2E2E5C2E2E5C2E2E5C2E2E5C6333
:10C210006F6D706F6E656E74735C6C696272617263
:10C220006965735C626F6F746C6F616465725C6486
:10C2300066755C6E72665F6466755F7665725F7662
:10C24000616C69646174696F6E2E63002E2E5C2EC2
:10C250002E5C2E2E5C2E2E5C2E2E5C636F6D706F0E
:10C260006E656E74735C6C69627261726965735C31
:10C2700074696D65725C6578706572696D656E7400
:10C28000616C5C6170705F74696D6572322E630001
:10C290002E2E5C2E2E5C2E2E5C2E2E5C2E2E5C63A3
:10C2A0006F6D706F6E656E74735C6C6962726172D3
:10C2B0006965735C74696D65725C657870657269D7
:10C2C0006D656E74616C5C6472765F7274632E630C
:10C2D000000000002E2E5C2E2E5C2E2E5C2E2E5C7E
:10C2E0002E2E5C636F6D706F6E656E74735C6C691F
:10C2F000627261726965735C6578706572696D659B
:10C300006E74616C5F6D656D6F626A5C6E72665FA4
:10C310006D656D6F626A2E63000000002E2E5C2E2C
:10C320002E5C2E2E5C2E2E5C2E2E5C636F6D706F3D
:10C330006E656E74735C6C69627261726965735C60
:10C340006578706572696D656E74616C5F73656345
:10C3500074696F6E5F766172735C6E72665F73652F
:10C360006374696F6E5F697465722E63000000000C
:10C370004E52465F4552524F525F494E56414C49CC
:10C38000445F4441544100004E52465F4552524F73
:10C39000525F534F46544445564943455F4E4F54B0
:10C3A0005F454E41424C4544000000004E52465FFE
:10C3B0004552524F525F464541545552455F4E4F8C
:10C3C000545F454E41424C45440000004E52465F8A
:10C3D0004552524F525F4D555445585F554E4C4F44
:10C3E000434B5F4641494C45440000004E52465F76
:10C3F0004552524F525F4D555445585F4C4F434B39
:10C400005F4641494C4544004E52465F4552524FAB
:10C41000525F4D555445585F434F4E445F494E4916
:10C42000545F4641494C4544000000004E52465F6F
:10C430004552524F525F4D555445585F494E4954ED
:10C440005F4641494C4544004E52465F4552524F6B
:10C45000525F424C455F495053505F52585F504BBA
:10C46000545F5452554E4341544544004E52465F2A
:10C470004552524F525F424C455F495053505F50B6
:10C480004545525F52454A4543544544000000002B
:10C490004E52465F4552524F525F424C455F4950A3
:10C4A00053505F4C494E4B5F444953434F4E4E45AA
:10C4B00043544544000000004E52465F4552524FDF
:10C4C000525F4150495F4E4F545F494D504C454D6E
:10C4D000454E5445440000004E52465F4552524F6F
:10C4E000525F4E4F545F535550504F525445440085
:10C4F0004E52465F4552524F525F4D4F44554C4548
:10C500005F4E4F545F494E495449414C495A454446
:10C51000000000004E52465F4552524F525F4D4F51
:10C5200044554C455F414C52454144595F494E4941
:10C530005449414C495A4544000000004E52465F60
:10C540004552524F525F4E4F545F464F554E440036
:10C550004E52465F4552524F525F494E56414C49EA
:10C56000445F5354415445004E52465F4552524F2A
:10C57000525F444154415F53495A45004E52465F11
:10C580004552524F525F494F5F50454E44494E47C6
:10C59000000000004E52465F4552524F525F5356C4
:10C5A000435F48414E444C45525F4D495353494EB9
:10C5B000470000004E52465F4552524F525F494E6F
:10C5C00056414C49445F4C454E47544800000000DA
:10C5D0004E52465F4552524F525F4452565F545737
:10C5E000495F4552525F414E41434B004E52465FB8
:10C5F0004552524F525F4452565F5457495F45521D
:10C60000525F444E41434B004E52465F4552524F9B
:10C61000525F494E5445524E414C00004E52465FC7
:10C620004552524F525F53544F524147455F465512
:10C630004C4C00004E52465F4552524F525F4E5591
:10C640004C4C00004E52465F4552524F525F494E8D
:10C6500056414C49445F504152414D004E52465F55
:10C660004552524F525F4E4F5F4D454D0000000006
:10C670004E52465F4552524F525F464F52424944D6
:10C6800044454E004E52465F4552524F525F44520F
:10C69000565F5457495F4552525F4F564552525567
:10C6A0004E0000004E52465F4552524F525F494E77
:10C6B00056414C49445F4144445200004E52465F4B
:10C6C0004552524F525F5245534F555243455300C6
:10C6D0004E52465F4552524F525F494E56414C4969
:10C6E000445F464C414753004E52465F53554343C7
:10C6F000455353004E52465F4552524F525F424C93
:10C70000455F495053505F4348414E4E454C5F4151
:10C710004C52454144595F45584953545300000019
:10C720004E52465F4552524F525F434F4E4E5F430B
:10C730004F554E54000000004E52465F4552524F36
:10C74000525F54494D454F55540000004E52465FCC
:10C750004552524F525F4255535900002E2E5C2EC7
:10C760002E5C2E2E5C2E2E5C2E2E5C636F6D706FF9
:10C770006E656E74735C6C69627261726965735C1C
:10C780006578706572696D656E74616C5F6C6F67FA
:10C790005C7372635C6E72665F6C6F675F64656624
:10C7A00061756C745F6261636B656E64732E6300A8
:10C7B0002E2E5C2E2E5C2E2E5C2E2E5C2E2E5C637E
:10C7C0006F6D706F6E656E74735C6C6962726172AE
:10C7D0006965735C6578706572696D656E74616CAE
:10C7E0005F6C6F675C7372635C6E72665F6C6F67C1
:10C7F0005F66726F6E74656E642E63007761726E31
:10C80000696E670064656275670000001B5B313B01
:10C8100033306D001B5B306D000000001B5B313B53
:10C8200033316D001B5B313B33326D001B5B313BA1
:10C8300033336D001B5B313B33346D001B5B313B8D
:10C8400033356D001B5B313B33366D001B5B313B79
:10C8500033376D00696E666F000000006572726F9D
:10C86000720000002E2E5C2E2E5C2E2E5C2E2E5C76
:10C870002E2E5C636F6D706F6E656E74735C6C6989
:10C88000627261726965735C6578706572696D6505
:10C890006E74616C5F73656374696F6E5F766172ED
:10C8A000735C6E72665F73656374696F6E5F6974E3
:10C8B00065722E680000000073645F626C655F63E0
:10C8C00066675F73657428292072657475726E657A
:10C8D00064202573207768656E20617474656D70BF
:10C8E00074696E6720746F2073657420424C455FD5
:10C8F00047415454535F4346475F5345525649435B
:10C90000455F4348414E4745442E000073645F62D3
:10C910006C655F6366675F73657428292072657450
:10C9200075726E6564202573207768656E2061746A
:10C9300074656D7074696E6720746F207365742000
:10C94000424C455F434F4D4D4F4E5F4346475F5608
:10C95000535F555549442E0073645F626C655F6395
:10C9600066675F73657428292072657475726E65D9
:10C9700064202573207768656E20617474656D701E
:10C9800074696E6720746F2073657420424C455F34
:10C9900047415454535F4346475F415454525F5498
:10C9A00041425F53495A452E0000000073645F62A4
:10C9B0006C655F6366675F736574282920726574B0
:10C9C00075726E6564202573207768656E206174CA
:10C9D00074656D7074696E6720746F207365742060
:10C9E000424C455F434F4E4E5F4346475F47415081
:10C9F0002E00000073645F626C655F6366675F733F
:10CA0000657428292072657475726E6564202573BB
:10CA1000207768656E20617474656D7074696E67E7
:10CA200020746F2073657420424C455F4741505F0E
:10CA30004346475F524F4C455F434F554E542E007F
:10CA400073645F626C655F6366675F7365742829F2
:10CA50002072657475726E65642025732077686531
:10CA60006E20617474656D7074696E6720746F20D8
:10CA700073657420424C455F434F4E4E5F434647BB
:10CA80005F474154542E00006170705F74696D659A
:10CA9000722E6D5F6466755F696E61637469766935
:10CAA00074795F74696D6572000000006170705F79
:10CAB00074696D65722E6D5F7764745F6665656419
:10CAC0005F74696D657200006E72665F626F6F748D
:10CAD0006C6F616465725F77647400006E72665F8C
:10CAE0006466755F626C650062616C6C6F632E6D6D
:10CAF0005F6275666665725F706F6F6C0000000044
:10CB00006E72665F6466755F666C617368000000D4
:10CB10006E72665F6466755F7265715F68616E6490
:10CB20006C6572006E72665F6466755F73657474BF
:10CB3000696E6773000000006E72665F6466755F01
:10CB400073657474696E67735F7376636900000060
:10CB50006E72665F6466755F76616C696461746944
:10CB60006F6E00006E72665F6466755F7665725FF9
:10CB700076616C69646174696F6E00006170705FEA
:10CB800074696D657200000061746669666F2E6D70
:10CB90005F7265715F6669666F0000006D656D5F4D
:10CBA0006D6E6772000000006E72665F6673746F70
:10CBB000726167650000000061746669666F2E6DC2
:10CBC0005F6669666F000000736F72746C697374DE
:10CBD0000000000062616C6C6F632E6C6F675F6DAC
:10CBE000656D706F6F6C0000617070006E72665FD3
:10CBF000736468006E72665F7364685F626C650080
:10CC00006E72665F7364685F736F6300020000009A
:10CC100000000000F9290F00A5290F0067E6096A46
:10CC200085AE67BB72F36E3C3AF54FA57F520E514D
:10CC30008C68059BABD9831F19CDE05BFFFFFFFF1D
:10CC4000FFFFFFFFFFFFFFFF0000000000000000EC
:10CC50000000000001000000FFFFFFFFFCFFFFFFDE
:10CC6000FFFFFFFFFFFFFFFF0000000000000000CC
:10CC70000000000001000000FFFFFFFF512563FCE2
:10CC8000C2CAB9F3849E17A7ADFAE6BCFFFFFFFF47
:10CC9000FFFFFFFF00000000FFFFFFFF000000009C
:10CCA00096C298D84539A1F4A033EB2D817D037746
:10CCB000F240A463E5E6BCF847422CE1F2D1176BE1
:10CCC000F551BF376840B6CBCE5E316B5733CE2BB4
:10CCD000169E0F7C4AEBE78E9B7F1AFEE242E34FE3
:10CCE000FFFFFFFF7F000000800000000000000049
:10CCF00000000000FFFFFFFF7F0000008000000039
:10CD0000000000000000000054CE0F00B8570020C3
:10CD1000C40100006C150F00B8CE0F007C59002034
:10CD2000A46F00000E2E0F003D430F0075430F004F
:10CD30001D380F0041370F0088CA0F0000000003A4
:10CD4000ACCA0F0000000003C8CA0F0000000404B2
:10CD5000DCCA0F0000000404E8CA0F000000000352
:10CD600000CB0F000000040410CB0F0000000404EF
:10CD700024CB0F000000040438CB0F000000040493
:10CD800050CB0F000000040464CB0F00000004042B
:10CD90007CCB0F000000000088CB0F0000000003D8
:10CDA0009CCB0F0000000000A8CB0F000000040483
:10CDB000B8CB0F0000000003C8CB0F00000000003C
:10CDC000D4CB0F0000000003E8CB0F0000000404E8
:10CDD000ECCB0F0000000303F4CB0F0000000303B3
:10CDE00000CC0F000000030318580020EC6D002059
:10CDF000FD6D0020006E002034590020F40000007A
:10CE0000C0580020B8580020C0580020AC8700202F
:10CE1000685900201800000011390F0000000000C0
:10CE2000A57E0F0000000000DD7E0F000000000066
:10CE3000318C0F0000000000BD8D0F0000000000CD
:10CE4000BD7E0F0000000000000000000300000095
:10CE5000DD6F0F00011C1324590218200A15281C2D
:10CE600012FF031CFFFF02340115100140110211D3
:10CE7000040A1954A0C1DA60280425F0BB0F145C21
:10CE8000C80F14FCC70F1A54081A04041A14041A01
:10CE90000C041A1C041A24041A2C041A34041A3C14
:10CEA000041A44041A4C04518490D0031B554614B0
:08CEB0003A10C5015900000011
:020000041000EA
:0410140000100F00B9
:020000041000EA
:0410180000E00F00E5
:04000005000F1201D5
:00000001FF
